:020000041100E9
:10300000002373B52B4D2C4C28006361022601F080
:103010005DFA4021FE2221742800284B009601F021
:10302000A7FA002836D1217CFF222800244B0096E5
:1030300001F09EFA00282DD1224BA2899A4226D176
:10304000E389214A93420DD1204B6361204B2268D2
:10305000002A03D1002B01D043CB43C4280001F048
:1030600073FA73BD1B4A934201D00023EFE71A4B5A
:103070001A4A1B68934206D9C02304222800217CE7
:103080009B0001F0EBFA114B6361154BDFE7002366
:103090002374EAE7CC233821AC2228009B01217459
:1030A00001F0DCFA0028F2D10E4B63610E4BE38194
:1030B0000E4BCCE7D443FF1F8063FF1F8C63FF1FC1
:1030C0008E63FF1F5959000083050000F94200116B
:1030D0002CBE001182150000A463FF1F871300009F
:1030E00038BE0011B1430011AAAAFFFF20BE001193
:1030F000F7B5164B0192C318021D002000938823D8
:103100005B05D3181B685C1C1AD09CB2402C18D8E5
:103110008D781E0CAC466746CD782D023D43AE42FD
:1031200006D1019800280ED110000C70240A4C70B2
:1031300003249BB20733A343D218009B9A42DED3E9
:10314000FEBD4432F9E71000FAE7C046FC0F00006C
:10315000802213B503000324019189B25201073183
:103160009B18A14304305A1A88235B05C3181B68B7
:10317000591C03D190429241104016BD99B240298A
:1031800007D80B000733A343C0189042ECD30020AC
:10319000F3E74430F9E7134B134A1B68126810B584
:1031A000FA24934201D81A00F824104BE4021B6859
:1031B0009A4210D813000E4A12689A420ED3013375
:1031C00007D1F823DB029C4203D10A49054808F0E5
:1031D000CBFA200010BDFC24E402ECE7FE24E4025C
:1031E000F7E7C04600C0071100D0071100E0071143
:1031F00000F00711FFFFFF7FF0B59BB015000490B2
:103200000391402A00D9A0E006AB59801A80FFF74D
:10321000C2FF0400042816D9002206A9FFF768FFA0
:10322000052810D906AB1B88AB420CD1002D07D066
:10323000514B2A000499C01808F02EFD002802D135
:1032400001201BB0F0BD06AB1D8020000699FFF7E2
:103250007FFF041E7BD1069B0793FFF79CFF802313
:103260005B01C618802307001B039E4201D3F8268A
:10327000F60288235B05F31801931B68013302D023
:10328000019808F049FC3D49019808F06DFA3B1D92
:103290000293331D05938822029B52059B181B68DD
:1032A00008935A1C3CD044219AB20091402A04D879
:1032B0000320D11D814389B2009103991B0C8B42DD
:1032C00024D0402A22D80122300008A9FFF710FF9D
:1032D000021E1BD1380008A9FFF70AFF04000428CA
:1032E00031D9009A059B9B1880225201B218934253
:1032F00040D288235B05C118009A09A808F094FA07
:103300001D4B009A09A9F01808F05EFC009A029B78
:103310009446634402931A4B029AFB189A42BAD31A
:1033200088235B05FC1821680198013908F01CFA14
:10333000200008F0F1FB039A07AB5A803000079990
:10334000FFF706FF0400002C03D1002079E70428D2
:10335000FBD988235B05E018069908F005FA0323DA
:10336000EA1C9A4300D16BE7034B0499E01808F07C
:103370002BFC65E70424ECE704000011FFFFFF7F4E
:10338000F80F0000F7B505001400402A21D80027E7
:1033900001AE71803780FFF7FEFE042816D93A008F
:1033A0003100FFF7A5FE042810D93688BC420BD0A7
:1033B000BD4209D0221CB44200D9321C064B92B245
:1033C000C118280008F030FA30B2FEBDC04300B288
:1033D000FBE703204042F8E70400001137B5042260
:1033E00004000D0001A81649FFF7CCFF02000428D5
:1033F0000BD1019BA34208D3AB4204D0104901A8D2
:103400000195FFF7F9FE01203EBD0E4C2368200018
:10341000019308F081FB019920000139019108F026
:10342000A3F980235B01E418074B9C42EED10422F0
:10343000034901A80195FFF7DFFE0020E4E7C0463D
:103440005555000000C007110000081130B589B0C3
:1034500008F01AFC10226946254808F035FB254B78
:10346000009A9A420ED1019B029A0F2B33D8002169
:1034700001240698013B08D2002900D00292029B49
:10348000013331D10023029325E0551CF2D1020013
:103490002100EFE710341022200004A908F014FBEB
:1034A000029B013301D1069B0293882304995B059B
:1034B000C918059B06981A03120B049105928142C4
:1034C00003D02B4201D108F0AFF9019B013B0193DE
:1034D000019B002BDED1029B002B03D004930498A8
:1034E0004168084709B030BDE025014C2D03EFE7E6
:1034F0000000011150485936F7B50F4F0F4BFA6DC8
:1035000004001A4084235B001343FB65030010335F
:10351000019300252E00112008F07EF90322BB6ED6
:103520001340AB4002351E43202DF4D1019B40C413
:10353000A342EED1F7BDC04600F0004000FEFEFF02
:10354000802270B5AD4CAE4BD200002120001C6033
:1035500008F04AFA2300AB4A88331A60AA4B1A785B
:103560006E23002A00D01133E3620A232365A74BA0
:103570001878A74BA0630138E361C3B2032B01D8CD
:1035800010232362A34B37226361C823DB00A361AE
:1035900023008C331A60082336210F3AE518E163C3
:1035A00023646264E9670439251DE96725003B2629
:1035B000BC352E602500C0352B602500C4352A603F
:1035C00025000636CC352E602500083EC8352E6015
:1035D0002500D03529602100D4310B602100D8317D
:1035E0000A6021000225E0310D6025004221DC3512
:1035F000296025001B3EE4352E602500E8352B6050
:103600002500EC352A6022000525F43215602200E1
:10361000F032116022001831903211602200943291
:10362000136023003C2298331A60AF23DB00236031
:10363000794B2363032805D808F04EFA3302353757
:103640001523636096232100FA225B00A360E360E8
:10365000C8332361714BFC319200A3640A6062623B
:103660006F4A704DA2627322E2656D3A6265A2658F
:103670000232E5644A600221616696218900A166F2
:10368000626709210022E166A2676749674A684EBE
:103690002167E2673560032811D808F01DFA960803
:1036A0009EA61023CDE70E23CBE70C23C9E720000D
:1036B0001A259C30056020000735A03005602000E9
:1036C000A83003602300FA20F8338000186023003C
:1036D0006420A433186023005F38AC3318602300E3
:1036E0000338B03318602300C630B43318602300A9
:1036F0000020B833186023003825FC339D604D4D01
:103700005A665D644C4D9A64DD619625AD001D627C
:103710004A4D9A675D62F53DFF3D9D621E25484A10
:10372000DD6618675867D9651966DA67BE23C02158
:10373000444A5B00E250444B4900635004316250FC
:10374000C4225200A350FA23E4205B000432A350A9
:103750000432A3503D493E4A3E4BD1603E49800071
:1037600019503E49E938FF3819503D490430195085
:103770003C491038D1613C4911633C4951633C4993
:1037800011603C49195019003B48F83108603B4929
:10379000D16582213A4A89005A501A0039490832C3
:1037A000D1671A003849B43211608821374A89003C
:1037B0005A501A00364988321160364ADA6408F0E5
:1037C0001BF9012008F010FA70BD200014259C3070
:1037D000056020000435A03070E7200010259C30E3
:1037E000056020000335A03068E720000E259C30DE
:1037F000056020000235A03060E7C0460004FF1FCE
:103800005C66FF1F5071FF1F1446FF1F4A0AFF1F0F
:103810003A07000080C3C9019A02000050C30000AB
:103820006A180000280A0000204E000088130000DB
:10383000F009FF1F001F001168100000C4090000FC
:10384000DC05000040420F0010270000FD1BFF1F99
:10385000FC00FF1F0000FF1F092FFF1F3132FF1F59
:10386000C930FF1FDD1FFF1FF91FFF1FA521FF1F0D
:10387000491FFF1FC928FF1F712CFF1FD918FF1FE9
:10388000D527FF1F3D25FF1F4925FF1F491EFF1F8D
:10389000011FFF1FC11DFF1FF7B50B0CFF270122E2
:1038A000009300233C001E001D009446019089B245
:1038B00062469A401000084018413618B6B2FF2FF1
:1038C00002D1012E00D19FB2009802401A41AD18DA
:1038D000ADB2FF2C02D1012D00D19CB20133102BCF
:1038E000E6D10320012E07D1012D04D1019B240133
:1038F000E4191C700138FEBD102EFCD10238102DC9
:10390000F9D00230F7E710B5064C2378002B07D129
:103910000548FFF7F1FD0548FFF7EEFD0123237091
:1039200010BDC0461C66FF1F3066FF1F2066FF1FCC
:10393000F0B58BB00D0001230190102936D8FFF7A8
:10394000E2FF00231A001B48C15C01335218102B00
:10395000FAD1023B002A29D0174B184C1F680023CC
:1039600006A9E25C1600FA5C56405E540133102B47
:10397000F7D102AA08F030F92A0002A9019808F04C
:10398000EBF808F0C9F923681B18236008F0C4F9A4
:1039900063681B18636008F0BFF9A3681B18A36075
:1039A00008F0BAF9E3681B18E360002318000BB0B5
:1039B000F0BDC0463066FF1FB444FF1F2066FF1FE6
:1039C0000223F0B501245D4D5D4E2B705D4B91B02F
:1039D0001C705D4F039333680820BB7006F036FC03
:1039E0000023984205D0BA78552A02D0332A00D055
:1039F00098E03360002006F0A9FE07F01DFFFFF7F6
:103A00009FFD07F059FF1F22012400214F4B10AEEC
:103A10001A704F4B1C704F4B19704F4B19689143E4
:103A2000163A0A431A60602219689143403A0A43E1
:103A30001A6008F0E1F808F0BFF8C120FF21474BF9
:103A400080001A588A431A50C52292009858884319
:103A5000BF39014399509858414908408021C90114
:103A60000143802099509958C0050902090A014371
:103A7000995080213B48490108F096F80323220021
:103A8000394901940093394808F05EF82C223849EE
:103A900005A807F0C9FE05AC61782078023406F06D
:103AA000F5FBA642F8D10121002006F003FD314BC1
:103AB000314A196803201140A022D2020A431A6039
:103AC0008022196892040A431A6019682B4A11402F
:103AD000802292030A431A60294B2A4A934200D853
:103AE000012007F0E1FD07F047FE07F0D5FF287839
:103AF00008F0F2F8039B1878C0B207F0FDFF07F05A
:103B0000DBFD2149042008F087F806F0EBFD00F00A
:103B1000AFF800F0F9FD00F08BFE00F019FA00207C
:103B200011B0F0BD00932100174A042007F054FEA5
:103B30008023DB059C62FFF789FC5BE74A0AFF1FD5
:103B400034F000401446FF1FB063FF1F480AFF1FF8
:103B5000490AFF1F680AFF1FBCF0004000E100E0B7
:103B6000FF00FFFF1846FF1F9C58FF1F1856FF1F3E
:103B700048BD001114F00040FF7FF8FFFFFF9FFFDA
:103B80005071FF1F0080FF1F3B00010870B500252A
:103B90002849294A29484D6308CA1B051B0DED1801
:103BA0008242F9D10022264B8B63264B08211A62F0
:103BB0008022254B9205DA67244BDA688A43DA6063
:103BC000234A1278012A03D09A6822490A409A604F
:103BD0000121EE242048E40002686C438A4302601D
:103BE000DA6811208A43DA6008F03EF8112007F005
:103BF00043FE112007F070FD184A200C04006423D6
:103C000090420AD8FA220023D200904205D9144BE0
:103C10000A21C01808F090F8C3B2124A1372124B6E
:103C2000D4801B78002B04D1104B1021187807F09A
:103C3000B3FE70BD00000540880505400006054044
:103C4000FF01000000F0004004E100E03CF0004013
:103C50004A0AFF1FFFDFFFFF00380040B70B0000DC
:103C600030F8FFFF9863FF1FD465FF1FD063FF1F6D
:103C7000002210B51100112007F0BEFD10BD00009C
:103C8000F8B5002301250826394F3A4C3B62E3681A
:103C90001120AB43E360E368B343E36007F0ECFD5E
:103CA000112007F0E1FF112007F05EFF402322689A
:103CB00029001343236080236268DB0213438022C0
:103CC0006360A36807201343A360A3682A4A1340D4
:103CD000A3608023A2689B0113431022A360236C7E
:103CE00093432364236C2B43236480235B003B6258
:103CF000226B224B1A402263626B1A406263A26BF2
:103D00001A40A263E26B1340E3631D4AE368134069
:103D1000E36006F0A1FB2900072006F0CBFB802121
:103D2000184A1120536C0B43536407F03DFEFD21EC
:103D3000154B164A89005A508023C720626B5B03DB
:103D400013436363E36880003343E360E368104A2E
:103D50001D43104BE56019581140802212020A439E
:103D60001A50802292051A600B4B5E63F8BDC04664
:103D700000F000403CF00040FFFFDFFFEFFFEFFFEF
:103D8000FFFF7FFF003800400000FF1F8D3B001148
:103D9000FF00FFFF00E100E00000054030B503A890
:103DA00004880B20002C0ED14968074D087849780B
:103DB000090201430A20A94205D1012120001980EE
:103DC000024B1B7A137030BD192A00009863FF1F45
:103DD000F7B5150008AA16884A680F4F147852786C
:103DE000120222430A24BA4214D10122DBB2019208
:103DF00000962A0007F0C6FB041E0BD1074B1B6878
:103E0000002B07D068782A780002104342425041C4
:103E1000013098472000FEBD022900001C63FF1FEF
:103E200030B5012503790400BFB02B4212D00A49F6
:103E3000408806F013FF28420CD06A46074B6946BB
:103E40005B8D55801380064B60881B7A13710022AE
:103E500003F0E4FF3FB030BD1463FF1F4842FF1F73
:103E60009863FF1F10B50549054806F0ADFE042113
:103E7000044A054806F06AFE10BDC0461463FF1FE1
:103E8000FFFF000074BD00114842FF1F10B502483B
:103E900004F046FE10BDC046213E0011062310B5B9
:103EA000837010330371443B43712A33837144336D
:103EB000C37100230222012103720E4B0270417074
:103EC0001C8881724472197A0273C1729A784273A3
:103ED000DA7882730322C2731A7902745A794274AF
:103EE0000C2282749A79C274DB7903751123C37032
:103EF000152010BD9863FF1F10B5142007F004FEB5
:103F0000124B14220021186007F06EFD002007F00C
:103F10009BFC012007F0C8FC022007F005FD0320F0
:103F200004F0A2F8042006F0B7F8052003F0E0FA48
:103F3000062003F0ADFF072001F0AEF9082006F0DF
:103F4000E5FD092000F088FF10BDC0462063FF1F7B
:103F500010B507F059FC012007F0CEFB07F00CFE6E
:103F6000002010BD094B10B50400984205D001296E
:103F700004D12000064906F027FE10BD0229FCD11D
:103F8000013904F08BFD0028F3D0F6E7FEFF0000B6
:103F90004663FF1F70B50D7A100004AA2C00168826
:103FA00010221440154220D1002E20D10A78022A76
:103FB00018D14A68517815780E4A0902294391426E
:103FC00005D00D4A914209D01C800A2404E0142235
:103FD0000A491A8007F028FC200070BD0C2208490D
:103FE0001A80F7E71C800124F6E70824F4E70B2485
:103FF000F2E7C046F3FF0000F4FF00009844FF1F03
:1040000050BE001110B504000749084806F0DCFD59
:10401000074804F0C5FC0020E40704D50721054A41
:10402000054806F093FD10BD4663FF1FFFFF00002B
:10403000653F0011B8BD00118C42FF1F00B50C4B4D
:10404000BFB01A780B4901A800F024FC6B4680B27F
:104050005880002809D06A46074B69461B881380A0
:10406000064B0022188803F0D9FE3FB000BDC046C1
:104070002463FF1F2563FF1FE642FF1FEE43FF1F60
:1040800000B50C4BBFB01A780B4901A801F00CFE2B
:104090006B4680B25880002809D06A46074B6946B3
:1040A0005B8D1380064B0022188803F0B7FE3FB0EB
:1040B00000BDC0464E63FF1F4F63FF1F8C42FF1FB2
:1040C000EE43FF1FF7B50E00377A1C0008AB110056
:1040D0003D001A8820231D401F423CD13378022B1B
:1040E0003BD173681F785B781B023B431E4FBB427A
:1040F00008D01E4FBB4214D01D4DAB4221D00A2523
:104100002800FEBD002A2AD1142C2AD82200F068EB
:1041100007F08AFB174B1C70012CF1D9FFF7B0FF99
:10412000EEE7002A1BD1202C1BD82200F06807F0F4
:104130007BFB114B04211C70104B187807F02CFCF2
:10414000DEE7E3B20124009201940A00310007F097
:1041500019FA0500D4E70825D2E70125D0E70B2599
:10416000CEE70D25CCE7C046F3FF0000F4FF0000CA
:10417000022900004E63FF1F2463FF1FD063FF1F4F
:10418000332310B5040003700A220749013007F0F9
:104190004BFB064B0F201B681A0AE37222731A0CA2
:1041A0001B0E6273A37310BD9863FF1FC063FF1FD4
:1041B00030B5012503790400BFB02B4213D00B4961
:1041C000408806F04BFD28420DD06A46084B01A8F6
:1041D0001B881380FFF7D4FF6B4658800022694686
:1041E000608803F01BFE3FB030BDC0464663FF1F32
:1041F000E642FF1F10B5024804F092FC10BDC04615
:10420000B141001170B5160004AA148805AA1578EA
:104210004A685078117800022A4A08438018052815
:104220004BD807F059FC03131E29343F0720032CF9
:104230000BD80422121BAA4200D92A0022491A8054
:104240003000091907F0F0FA002070BD0720112C8A
:10425000FBD81222121BAA4200D92A001B491A803D
:10426000EEE707200E2CF0D80F22121BAA4200D92D
:104270002A0017491A80E3E70720032CE5D8042217
:10428000121BAA4200D92A0012491A80D8E7072037
:10429000032CDAD80422121BAA4200D92A000E49A4
:1042A0001A80CDE70720032CCFD80422121BAA4284
:1042B00000D92A0009491A80C2E700220A201A8080
:1042C000C3E7C046DCD5FFFF03BE00116C63FF1FD0
:1042D000F3BD0011EEBD0011E9BD0011E4BD0011F8
:1042E00010B50D21024A034806F030FC10BDC0464F
:1042F000D8BD0011FC42FF1FF0B50024274E85B049
:104300003000B47100F0E2F8254D264BEA89297C93
:104310009A422FD10423300003AA00F057F9040079
:10432000300000F011F90123B371002C34D16B4639
:1043300099892B68C9BA4B4329891B4A1B145B18FE
:1043400053806B46D9896B6849BA89B24B436989F6
:104350001B0C5B181548191C1BB2834200DD011CA5
:104360000B0400D5002113889180013313802000B5
:1043700005B0F0BD0227220003AB3000009700F02B
:10438000F7F80E230400297C0122300000976B44CB
:1043900000F0EEF80443C3E71C00E8E7D443FF1F36
:1043A0008063FF1F830500009863FF1F0F27000035
:1043B00073B5234E300000F089F8224D07236A467A
:1043C0003000297C00F002F904003000002C33D1C9
:1043D0006B461B787F2B2FD800F0B6F86B46D87849
:1043E000F02302041B031A406B469B8816495BBAF4
:1043F0009BB21A432B68000953432A891B0C9B1854
:104400004B806B465A789B7812031B011A436B68EA
:10441000024353436A891B0C9B180C481A1C1BB29D
:10442000834200DD021C130400D500220B888A8021
:1044300001330B80200076BD00F086F80124F9E7F7
:10444000D443FF1F8063FF1F9863FF1F0F270000E7
:1044500070B5114C237C002B0FD0382B0ED10F4D93
:10446000280000F033F8CC23AC222800217C9B01EB
:1044700000F0F4F8280000F067F870BD084BE289FE
:104480009A42FAD1054D280000F020F800222800B9
:10449000217C00F0C5F8EDE78063FF1FD443FF1FC8
:1044A0008305000010B5084B1A7C002A09D05B690F
:1044B000002B06D09847041E01D0FEF7A1FD200076
:1044C00010BD0124F9E7C0468063FF1F70B5C179B4
:1044D00005000C00631E9C411A4BE402E4184900DD
:1044E0000460C9B2007906F01BF8E97968794900DF
:1044F0000131C9B206F014F8E8790930C0B207F00A
:1045000033FB0023E36661332360AA795B3B002A17
:104510000ED022689A43023B134323600A23E361CF
:104520000733236200232363A3630133E36370BD76
:1045300022689A43022313432360462363610633B0
:10454000A361EFE70050004070B500250400036848
:10455000DD66C0790930C0B207F08EF929002079F4
:1045600005F07AFF2900607905F076FF70BD000044
:10457000F8B51E0006AB1D78002304681700E3663B
:10458000616007F081FB01238022E3662B00276135
:104590005200013B08D207F05FFA08200A4A11686E
:1045A000002D03D12800F8BD2261F2E7236F0342FA
:1045B00003D02369013D3370013613685B1A032B66
:1045C000EED90125EEE7C0466008FF1F70B51C005C
:1045D000002305681600EB66696007F055FB0123B0
:1045E0008022EB6623005200013B08D207F034FA28
:1045F00008200A4A1168002C03D1200070BD2A61EE
:10460000F2E72B6F034203D02B69013C3370013674
:1046100013685B1A032BEED90124EEE76008FF1F35
:10462000002370B504681500E366616007F02CFB99
:104630000123E366256107F00FFA8020064A800017
:104640001168636B034205D113685B1A032BF8D919
:10465000012070BD0020FCE76008FF1F70B51D0041
:10466000002304681600E366616007F00DFB012378
:10467000E36626610F33626B1A42FCD02B0A23617A
:104680001023626B1A42FCD0EDB2256107F0E4F909
:104690008020074A80001168636B034205D11368CC
:1046A0005B1A032BF8D9012070BD0020FCE7C0463F
:1046B0006008FF1F70B51E00002305681400EB663C
:1046C000696007F0E1FA0123A619EB660F33B442E3
:1046D0000ED107F0C1F980200A4A800011686B6B87
:1046E00003420CD113685B1A032BF8D9012070BD6B
:1046F00021782961696B1942FCD00134E7E7002079
:10470000F5E7C0466008FF1F10B5084CE368002BB2
:1047100008D1074B1B685B045B0C0A336360054BD5
:104720001B68236007F008F9A06010BDC063FF1F7D
:10473000C8F00040CCF0004010B507F0A5FA0F4BD0
:10474000996A9A6A8A42FBD10D4C6268A0688A18FD
:10475000121A531E884200D31300A1602168DA0B9D
:1047600052185B0407495B0C636022600B60064BC8
:104770001A6007F071F9206810BDC04600F00040D3
:10478000C063FF1FC8F00040CCF0004070B51F4C64
:1047900023793F2B01D93F2323711D4B22791A70B6
:1047A0001878C0B207F0A0FA18231A491A4A0B80E9
:1047B0001A4913800B805380A379194980200B80FC
:1047C0000C21938001334B430001191C834200D913
:1047D000011C144BD18019806379002B11D1013356
:1047E0006371237A012B01D8022323726279237A21
:1047F0000D4853430A21584307F09EFA0B4D286099
:1048000070BDA02BEDD9A023EAE7C046B463FF1F1B
:10481000480AFF1FEC43FF1FC045FF1FEA43FF1F6D
:10482000A065FF1FE843FF1F71020000A463FF1F84
:10483000F8B513210020FEF7D1FD114C011E114DDA
:1048400009D10C22104BC1CBC1C4280007F0CCF811
:10485000FFF79CFFF8BD0C2220000C49FEF792FDEB
:104860000C2802D0084B43CB43C40C222800084933
:10487000FEF788FD0C28EBD00C220021E5E7C046AE
:10488000B463FF1F8063FF1F44BE0011FC0C0000D7
:10489000F50C0000F0B5002504000E0085B0AA421A
:1048A00068D04B1C087801934B78897837790902D6
:1048B0001943F3783F061B040B431F4303972070F3
:1048C0006570262800D190E01CD8102812D806F078
:1048D000CBFF4B00FE003100310031009600A400F8
:1048E0009D003100310031003100310031003100D4
:1048F0003100E400232800D1BEE025285DD0FF234D
:10490000637099E0602800D1A1E00AD8552834D01E
:1049100056284CD03328F2D12000FFF731FC050097
:1049200028E0722800D189E0DC2800D1EEE071286F
:1049300000D179E0DB2800D003E1042ADFD910257B
:10494000052A05D0551F2A003800711D06F06CFF9E
:1049500005223100200006F067FF2A003900601DA3
:1049600006F062FF053505E00C2220008B4906F0B9
:104970005BFF0C25280005B0F0BD013A884D0C2ADC
:1049800013D8002A0AD02800019906F04DFFFFF73E
:10499000FDFE0C2228008349FEF72EFC29000C2284
:1049A000601C06F041FF0D25E4E70C22EBE77C4D8F
:1049B0007D4B2A0043CB43C2E9E7013A7B4D0C2AE9
:1049C00011D8002A08D00199280006F02DFF0C22EA
:1049D00028007749FEF710FC29001322601C06F01E
:1049E00023FF1425C6E70C22EDE7704B29001322A4
:1049F00018001D0006F0F8FFFEF702FBECE70522A9
:104A00006C49601C06F010FF0625B3E712226A49C4
:104A1000601C06F009FF1325ACE708226749601CFB
:104A200006F002FF0925A5E77178F72900D966E7A6
:104A3000634B188801F094FD02259BE7614B012A26
:104A400003D072785A706270F6E75B7858E7013AE3
:104A50005D4D062A0ED8002A05D00199280006F0DF
:104A6000E3FE01F053F829000622601C06F0DCFE8C
:104A700007257FE70622F0E7042A04D9534D2F606B
:104A800006F05AFFA860FFF757FE0422039003A91F
:104A9000601C06F0C9FE05256CE74D4D062AE2D9DB
:104AA00006222800019907F0F7F80028DBD006223B
:104AB0000199280006F0B8FE062246492800FEF7B4
:104AC0009BFB01233F4A51780B435370CBE7931E66
:104AD000414F1A2B04D87378002B09D100F030F91C
:104AE0003E4B39001D78601C6A1E06F09DFE41E7B2
:104AF000551E2A000199380006F096FE3849AAB2E0
:104B00003800FEF779FB00F051F9E9E7022A00D8F6
:104B1000F5E67378BFB26370B378A370032A05D04B
:104B2000033A390092B2F01CFEF766FB10223900FE
:104B3000E01CFEF727FCC51C002800DB1AE76070AC
:104B40007AE7DA281DD1042A00D8D8E6082A15D930
:104B5000B37972791B021343F27912041A43337A40
:104B60001B0613433B603B68052231002000039382
:104B700006F05AFE0422601D03A951E7FE2363706C
:104B8000F1E7DE2800D0BAE6511E012A01D1002546
:104B9000F0E6019800F0A0FFF9E7C04650BE001112
:104BA000B463FF1FFC0C000044BE00118063FF1FB4
:104BB000F50C00008C63FF1F6C63FF1F3445FF1F63
:104BC000EE43FF1FB063FF1F8944FF1FC063FF1F39
:104BD0006509FF1FADAC0000B365FF1FB165FF1F86
:104BE000AEDE000070477047020010B5094B0A3274
:104BF000094C92B2DA815A8298811882207802F0A8
:104C000015FB0422054B012120781A7006F0C4FE22
:104C100010BDC046BE44FF1FFE65FF1FFD65FF1FA0
:104C2000013870B5042809D806F056FF0309280892
:104C30001200234B0221187806F0AEFE70BD204B07
:104C40000821187806F050FE00221E4B1A72F5E774
:104C5000802200241B4B1A4D52001A8108211A6829
:104C60002878DC7206F088FE2100287806F0CCFF58
:104C7000012000F069FE00F049FFDFE7104B08213A
:104C8000187806F031FE1048FFF708F90F4B104A6C
:104C90009B79002093800F4A13808022094B520099
:104CA000D8721A8100F050FE00F030FF0A4B5B789A
:104CB000002BC3D0094A136007F036F8BEE7C046A0
:104CC000D063FF1FA463FF1FF743FF1FB463FF1FE1
:104CD000C045FF1FA065FF1FB063FF1F34F00040F9
:104CE00010B501290BD1082809D1054B1B78002BE1
:104CF00005D02622034B04485A72FFF775FF10BDFA
:104D0000D465FF1FA463FF1FC40900000300F0B5B2
:104D10000A4D8E18B14202D152008018F0BD0C78B5
:104D20002F6824093C5D0F271C700C7801313C4032
:104D30002F683C5D5C700233ECE7C046E443FF1F24
:104D40000D22114B10B51A700C23104C1049237012
:104D5000093A033B0F48637006F066FD2D230122DC
:104D60000D490E48A371FFF7D1FF01220C49FFF74F
:104D7000CDFF01220B49FFF7C9FF00220A491000AD
:104D8000FEF73AFA10BDC046D065FF1FB165FF1FA0
:104D900003BE0011B365FF1F6709FF1FB865FF1F42
:104DA0006609FF1F6509FF1FAEDE000070B5124CDB
:104DB000132220001149FEF7E5FA114D002817DDF6
:104DC000AB78002B14D0431C2B7009236B7000238D
:104DD00000190370287829000130C0B206F0F4FDF4
:104DE000297822000139C9B2002005F0CDFD70BD3F
:104DF000FFF7A6FFEEE7C046B365FF1FAEDE00007B
:104E0000B165FF1F10B5114B1A781870002A0ED02B
:104E100000280BD10E4B1A78062A07D85423D3400A
:104E2000DB0703D50B4B187802F000FA10BD002801
:104E3000FCD0074B1B78012B02D0033B022BF5D88B
:104E4000044B0121187806F0A7FDEFE7D465FF1F9A
:104E5000FD65FF1FFE65FF1F70B5514E514A524957
:104E60003070082005F01CFC0121022005F022FB17
:104E7000022005F003FC0121002005F01BFB0020AF
:104E800005F0FCFB00F0ACFEFEF7BAF806F034FDCE
:104E9000032246494648FFF739FF2D240300042228
:104EA0001C7044490130FFF731FF30230470424D3C
:104EB000424C437083702E3B062220004049EB8712
:104EC000FEF760FA062813D0200006F0C5FC022881
:104ED00009D00321200006F0F7FC8D23E3706E3B20
:104EE000237119336371062220003549FEF784F9D6
:104EF000344B1B68FC335C64FFF758FF0020FFF75E
:104F000081FF314C314A0121314B1278207802F077
:104F10004FF9304A304B12780021207802F048F9DE
:104F200001222E4B1A702E4B9B78552B31D12D4BD5
:104F30003B325A722C4B2D4AAB81EA812B826A821A
:104F40002021307806F008FD0120404205F068FD80
:104F50000120404205F004FEFFF7C2F9FEF782FF90
:104F600000F0A6FC01204042FFF74CF8012006F0BB
:104F700013FCF72001F0D8FA0121307806F00CFD7F
:104F8000307802F0AFFA1A4806F0FEFBFEF778FE22
:104F900070BD6422174B5B7953431A000A32CBE78A
:104FA000D063FF1FE54B0011E14C00113445FF1F9A
:104FB0006C63FF1F8C63FF1FBE44FF1F6509FF1F4B
:104FC000ADAC00005C66FF1FFE65FF1F1644FF1FAF
:104FD000F743FF1FD065FF1FB165FF1FA265FF1FCD
:104FE000B063FF1FA463FF1FC4090000CE090000C7
:104FF000D263FF1FB463FF1FF8B50A0020230D0022
:105000001A40194257D0574B1B78002B50D0FFF74E
:1050100093FB554B554C564E99686268737A8A1AC1
:10502000DB039A4202D36160FEF72AFE327A217ACC
:10503000531EDBB2994205D1FFF70AFA002000F0B7
:105040009BFD0FE09142F9D300232372FFF72AFA68
:10505000012000F091FD474F3800FEF71FFF390097
:1050600006F052FB637A002B1FD0013BDBB2637268
:10507000002B1AD1404B9B78552B01D106F054FEE2
:10508000E37A002B0CD000233C4A3A4FE37213889A
:10509000380001331380FEF701FF390006F034FBBE
:1050A000642370795843FFF79FFD237A01332372FD
:1050B00020206840F8BD0BB2002B0ADA304B18787C
:1050C00006F0F2FD002801D006F0D6FC8020000298
:1050D000EFE70224214206D0244B01201A72FFF789
:1050E00091FE2000E5E70B071ED5FFF725FB1E4BC1
:1050F0001E491F4C98684A68637A821ADB039A42F9
:1051000002D34860FEF7BCFDFFF7CCF9FFF7A0F92A
:10511000012000F031FD00F0E5FB2368DB0701D53D
:10512000FFF768F80820C4E71024214206D00D4B91
:105130001B78002BD5D1FEF7A9FED2E7012421422E
:1051400007D0104800F06CF806F066FC00F0FAFC9E
:10515000C7E70424080020402142ABD0FEF76EFFD1
:10516000BFE7C046D465FF1FC063FF1FA463FF1FD6
:10517000B463FF1FF743FF1FB063FF1F9863FF1F58
:10518000D063FF1FDC43FF1FF0B51B4B1B4F1B8879
:105190003A8804001A4E1B4D85B09A420DD83288C9
:1051A0009A420AD3184B1A882B889A4205D1174A7B
:1051B000174B12881B889A421BD0052001F00AFA6F
:1051C0003B8802AA13803388019053802B88114DAD
:1051D00093800F4B02A91B88D3800F4B2A78188825
:1051E00002F026FF0D4B08212878019A1C7006F06A
:1051F0008BFB05B0F0BDC0469E65FF1FEC43FF1F53
:10520000EA43FF1FA065FF1F9C65FF1F9A65FF1FF4
:10521000E843FF1FFE65FF1FEE43FF1F9865FF1F5A
:1052200013B50C4B1C78002C11D1002801D00A4B6F
:1052300018600A4A0A4B11780A4A10780A4A019201
:105240000A4A0092002205F097FA200016BD1124A8
:10525000FBE7C046FD65FF1F9465FF1FFC65FF1F50
:10526000EC65FF1FFE65FF1FD865FF1FDC65FF1F94
:1052700010B5064B12201B78052B06D1044B1322C8
:105280001988044B187801F081FB10BDFD65FF1FE4
:10529000EE43FF1FFE65FF1F10B500240122114BD6
:1052A00052421870104B1C70104B1A8002F01AF901
:1052B00004220F4B21001A700E480C3206F0ECFA53
:1052C000102221000C4806F0E7FA07220B4B1C6065
:1052D0000B4B1C700B4B1C700B4B1A700B4B1C7048
:1052E00010BDC046FE65FF1FFD65FF1FEE43FF1F9B
:1052F000FC65FF1FEC65FF1FDC65FF1FD865FF1F06
:10530000B065FF1FAF65FF1FF043FF1FAE65FF1FB6
:10531000F8B5174C0600257806A814240078052D4A
:1053200023D1B41F134FA5B21824BD421DD88D1F21
:10533000ADB2BD4219D8FA256D00AA4215D21D00A2
:105340000D4F0A3DADB2BD420FD80C4C26800C4C1F
:1053500021800C4900240A800B4A1380FFF714FFB8
:105360000A4B0421187806F0BFFA2000F8BDC046A9
:10537000FD65FF1F790C0000750C0000EC43FF1F5A
:10538000EA43FF1FA065FF1FE843FF1FFE65FF1FE5
:10539000F0B50BB20D0089B0002B00DB70E1A44E1C
:1053A000307806F081FC041E50D00378A22B00D187
:1053B00022E1D02B1AD0912B45D143780E2B42D12C
:1053C0009C4B82889A423ED19B4A83681278052A78
:1053D00039D1032018567F2835D0984B1B68002BF5
:1053E00031D05B68002B2ED098472CE080780728BE
:1053F00029D806F071FB0428183F3F74A8D86378B9
:10540000002B0CD101218C4B19708D4B1A78002A7E
:105410005BD08C4B307801F0CBFE002855D00722B2
:10542000854B1A7051E061780029F8D1E378002BA0
:1054300011D0854A854B1278307801F0B9FE607042
:105440006378002BEBD1200006F016FB80200002D1
:10545000684009B0F0BD784B1B78022BF3D00121D6
:10546000307806F0E1FA0028EAD10121307806F020
:1054700093FAE5E76378002BD1D16F4F032807D16A
:105480003B78052B02D101333B701EE00223FBE782
:105490006F4B1A886F4B0293002A0BD01B78002B9E
:1054A00003D00121307806F02FFA3B78062B04D187
:1054B000013BE9E7029B1A70F7E7042B41D1012178
:1054C000029B3078197006F067FA5C4B1B68002B62
:1054D000B9D01B68002BB6D0574A107884E76378A0
:1054E000554F002B27D10622211D5B4806F09CF961
:1054F00062895A4B5A491A80A2895A4B1A80E38909
:105500000B800521397058490A80584A1380228A35
:10551000574B1A80574B1B78012B09D11F2001F0E4
:1055200059F8FA22920042430421307806F0ECF94F
:105530000022484B75E7312B00D070E70022454B25
:105540001A700323A0E706220021434806F0A4F9BD
:105550000023454A04211380444A30781380444A8A
:10556000138006F0C1F90821307806F0BDF9A3795F
:10557000083B5A425341304A03331370304B1B7877
:10558000002B06D0334B30781A78002A06D001F071
:105590004DFE0122314B52421A8096E701211970CB
:1055A00006F0FAF9F5E70821307806F09DF96378FE
:1055B000002B00D047E72C4B2D4F0293E388029A33
:1055C00004211380294B307803932389039A138095
:1055D00063893B8006F028FA002800D033E7264B89
:1055E0001B68002B00D12EE7039902983A8809889E
:1055F00000881B68984726E74379132B00D022E7E1
:105600000389012B0AD11D4B1B78022B06D10821DF
:10561000307806F069F9FFF72BFE14E7052000F05B
:10562000D9FF08210200307806F06EF90BE7C0467A
:10563000FE65FF1F05140000FD65FF1F9465FF1F39
:105640001644FF1FF743FF1FD065FF1FB165FF1F03
:10565000D265FF1FD465FF1FA365FF1FEE43FF1F29
:10566000AA65FF1FAC65FF1F9E65FF1F9C65FF1F9E
:105670009A65FF1FA265FF1F9065FF1F9865FF1FBA
:105680008020C001014200D0E2E6CB0731D5324B89
:105690001B78002B1DD0314E05AC3378052B1AD169
:1056A000023B23702E4B21001B7823722D4B1B785D
:1056B00063722D4B187801F01FFD002809D00720D8
:1056C0002A4B30701B68002B03D01B68002B00D0C6
:1056D00098470120BCE60E20254B06221B78254961
:1056E0002370254B1B78637002ABC01806F09CF842
:1056F000D8E7022308001840194209D0174B1B783D
:10570000052B03D11D4B188805F0DEFF02209FE614
:105710000424214203D0FFF737FD200098E6082338
:1057200008001840194200D193E6154B1C78012C53
:1057300003D0022C0DD008208AE6124B124A1349DE
:1057400013481B881288098800880094FFF7E0FD41
:10575000F1E7FFF78DFDEEE7D465FF1FFD65FF1F45
:10576000F043FF1FAE65FF1FFE65FF1F9465FF1F1F
:10577000B065FF1FF143FF1FAF65FF1FEE43FF1F23
:105780009865FF1FE843FF1FA065FF1FEA43FF1F47
:10579000EC43FF1F10B502A804880B20002C10D189
:1057A000496808784978090201430C48814209D1C7
:1057B000022119800A4B59881170DB7800205BB2F6
:1057C000537010BD074C0A20A142FAD10221198062
:1057D000034B998811705B79F0E7C0466E2A000090
:1057E0009863FF1F6F2A0000F7B5150008AA1688F6
:1057F0004A680F4F14785278120222430A24BA42A0
:1058000014D10122DBB2019200962A0005F0BAFE03
:10581000041E0BD1074B1B68002B07D068782A7831
:105820000002104342425041013098472000FEBD23
:10583000022900001066FF1F30B50125037904001E
:10584000BFB02B4227D01549408805F007FA2842FF
:105850000DD06A46124B69465B8D1380022353803C
:10586000104B5B8893806088002202F0D7FA0E49C3
:10587000608805F0F3F9C0070DD56A460B4B694601
:105880001B88138002235380064B9B88938060887B
:10589000002202F0C3FA3FB030BDC0460866FF1FC9
:1058A0001844FF1F9863FF1F0066FF1F7244FF1F0D
:1058B00010B5074C0749200005F086F9200006497D
:1058C00005F082F90721054A054805F03FF910BDAA
:1058D000FFFF00000866FF1F0066FF1FD0BE00111B
:1058E0001844FF1F10B5024803F01AF910BDC04656
:1058F0003958001170B55F25082607498400CA7819
:105900008B7840012A40B3433440A84323430243E9
:105910008B70CA7070BDC0468944FF1F010043B23E
:1059200004205A0002409B000C3003401A43152308
:1059300010B5044CE0789843143B0B4018430243E5
:10594000E27010BD8944FF1F10B5054B082419797A
:105950000A00A243002801D022000A431A7110BD98
:105960008944FF1F10B5054B4024D9780A00A24393
:10597000002801D022000A43DA7010BD8944FF1FBD
:105980000821F8B5324D334BAE7804000E40AE70AE
:10599000984204DD67232B70473B6B70F8BD2E4B9C
:1059A000984203DAE0232B703A3BF6E700232B7092
:1059B0006B7083B21A0029485F3292B2284F82423C
:1059C0002CD9002C03DA5B421CB204232B70053463
:1059D00020B20A2106F0B0F904B2FA239B009C42DF
:1059E00032DB08232A7813432B706421200006F051
:1059F000A3F90A2100B205F08FFE09B22A787B5C78
:105A000013432B700A21200006F096F90A2100B2F8
:105A100005F082FE09B27B5C6A780AE06970002CAE
:105A2000DBDA5B421CB204232B70F3226B78092C67
:105A3000E8DC13436B700A21200005F06DFE09B20B
:105A40007B5C1E43AE70A9E7632CCEDCEDE7C0465D
:105A50008944FF1F1B4E00001DFCFFFF2A080000A9
:105A6000FABE00110823F7B5194FCD003E790400A6
:105A70001E403E71EDB2632806DD5F3333433B7158
:105A800020231D437D71F7BD0300093305DA202370
:105A90005B4233433B71A623F3E70E4B019300288F
:105AA0000BDA0423444224B23B710A21200005F0A2
:105AB00033FE019B09B25B5CE3E70928F5DD0A21AF
:105AC00006F03AF9019B00B21B5C1E433E71ECE705
:105AD0008944FF1FFABE0011F8B50A4F05003B7854
:105AE0000E00002B0CD0084C2000FEF7EFFC33001A
:105AF0002A0020003978FEF7DDFD2000FEF724FDA6
:105B0000F8BDC0461B66FF1F9044FF1F70B50A4ECC
:105B10000A4D06223100280006F0BEF8002809D000
:105B2000074C31000622280005F07EFE07212000E8
:105B3000FFF7D2FF70BDC0468944FF1F1566FF1FE7
:105B40001466FF1FE622402110B50A4B1A70403A36
:105B50005A703E329A70DA780A40DA70082219795F
:105B60001140053A0A431A7197225A71FFF7CEFF86
:105B700010BDC0468944FF1F10B500282AD0164C1E
:105B80000A210223E05E06F0D7F800B2FFF7F8FE24
:105B90000423E05E642106F0CFF8012100B2FFF794
:105BA00061FF237A0024132220009A426041C0B290
:105BB000FFF7D8FE0320FFF79DFE2000FFF7AEFEA3
:105BC000064B1878053843425841C0B2FFF7BCFE77
:105BD000FFF79CFF10BDC0469863FF1FFD65FF1FC8
:105BE00070B500250A4C2000A571FEF76FFC10234C
:105BF0003E212000074AFEF75DFDA84200D13E3558
:105C0000054B20001D70FEF79FFC0123A37170BDA2
:105C10009044FF1FEABE00111B66FF1F0200F0B593
:105C200001270A480A4E51188B1A002B00DCF0BDE0
:105C3000082415784308684038404000805B013CE8
:105C400058406D08002CF5D10132EDE7FFFF000050
:105C50000ABF0011F0B500250F269D4200DBF0BD04
:105C60004C5D070944403440A400A05801357840F9
:105C7000F3E70000F0B589B06A460D000B000F276E
:105C8000110010351C780133260024093E4016709F
:105C900054700232AB42F5D12023024AFFF7DAFFFB
:105CA00009B0F0BD10BF0011F0B54E780B7889B087
:105CB00036020C00170001901E43012A61D9954B52
:105CC0009E4200D877E001339E421CD1062A17D1AC
:105CD000CA788B7812021A430B791B0413434A7952
:105CE00012061A438C4B5A6100221A705A808B4A52
:105CF0005A608B4A9A608B4ADA60002009B0F0BD86
:105D000088225205EEE7884B9E423CD182498B782F
:105D1000002B00D0F6E00C2A31D10F22A378934358
:105D2000E2781202134322791204134362791206B5
:105D300013434B60E279A07912020243207A0004F7
:105D40001043627A12060243CA60E27AA07A120213
:105D5000024376484A81834208D804236E491422BC
:105D600001980B7005F060FD1420C7E71201D218EE
:105D700089235B059A42F0D801238B70BDE7022A84
:105D8000FAD00523EAE76A4A01239642E6D1FFF7F3
:105D90006FFA052F0CD9E378A2781B0213432279FE
:105DA00012041A4363791B061343624A0393136078
:105DB00005F0BAFFA1E7584D2B78002B9DD1AB78A9
:105DC000002B00D1A0E02B8901339BB20093B3429A
:105DD00000D091E0132AD4D9CF7C8B7C3F021221D2
:105DE00020001F43FFF71AFF874200D08EE0002EED
:105DF0003DD1E378A2781B0213432279E9681204AB
:105E00001A4363791B06134303930A228B4212D170
:105E1000FF23A370E370237163716B89002B09D199
:105E2000E37B227C1B0212041343A27B13431B0956
:105E300001336B8100226B89002B8ED0002A67D141
:105E4000686837013818000B6B69000303909842AB
:105E500005D9686105F060FEEB780133EB70686886
:105E60001022A11C381805F0AFFE2E8145E76F897E
:105E7000009A7B1E9BB293423AD1E278A378120239
:105E80001A43237905A81B04134362796C68120630
:105E90001A43EB6800920392211D0C22049305F033
:105EA000C3FC0120260004A940421036FFF7E2FEA1
:105EB000013F012F17D1009A0B232861824200D0A5
:105EC0004CE704221C49200005F07EFE042203A9B1
:105ED000686805F071FCE968039AFF23914200D1DC
:105EE0003CE7F73B3AE73100FFF7C4FE1036DFE747
:105EF0000923B742A4D831E7009BB34200D9FCE69E
:105F000007232BE7022329E7032327E7062325E7B7
:105F10000A2323E7FFFE00009844FF1F0000011141
:105F2000FFFF00005048593601FF0000FFFF00113D
:105F300002FF000034F00040A444FF1F10B5034CE2
:105F40000B000122210000F06BFA10BDFD60001172
:105F50000B8870B506000D000224162B11D92B00FA
:105F60000322094900F05CFA041E0AD1074B2A8873
:105F70001B88191C934200D9111C300089B200F013
:105F8000EFFA200070BDC046296100117666FF1F40
:105F900010B54A780400013A0B000220012A07D804
:105FA0000A78002A04D005222000024900F038FABD
:105FB00010BDC046576100110A7810B50B000400EF
:105FC0000220002A04D007222000024900F028FA0B
:105FD00010BDC046036200110A7810B50B00040022
:105FE0000220002A04D009222000024900F018FAF9
:105FF00010BDC0466962001110B5034C0B000B22A6
:10600000210000F00DFA10BD9962001110B5034C8B
:106010000B000D22210000F003FA10BD0B630011EC
:1060200010B5034C0B000F22210000F0F9F910BD50
:10603000656300110A7810B50B0004000220002AE5
:1060400004D011222000024900F0EAF910BDC04638
:1060500075630011002310B51322190000F0E0F958
:1060600010BD000010B5034C0B001722210000F0FA
:10607000D7F910BDC7630011002310B5192219000C
:1060800000F0CEF910BD000010B5034C0B001B2230
:10609000210000F0C5F910BD01640011F7B5848935
:1060A0000D0006000121002C22D000238268D35667
:1060B0001778002B1EDA0C2C1AD90C3CA4B2131939
:1060C00040880093230002F086FE431E9841013071
:1060D0007B06DB0F6B703F23013C1F40A4B228708E
:1060E000AF70AC80002C07D0B3680133AB600021E7
:1060F0000800FEBD0020EBE7AC60F8E70B7803700A
:106100004B8843704B881B0A83700B79C370042043
:1061100070470420022B06D10020537811781B020F
:10612000009A0B43138070470B8803700B881B0A7F
:106130004370022070470420009983420AD15378AB
:1061400010781B0203430B80D37890781B02034323
:1061500000204B807047F8B50D004B7801240021DA
:10616000461C03702B788B4201D82000F8BD6B7859
:10617000B01C4F1C012B10D1890069184B880222DA
:1061800033704B88B9001B0A7370691805F0E4FC82
:1061900004360434A4B2F9B2E4E7122359436B186D
:1061A0005A88043132705B8810221B0A7370691898
:1061B00005F0D2FC12361234ECE770B5049D1400E1
:1061C0001E00052B01D8042070BD637812781B02D5
:1061D00013432B80E378A2781B02134302226B80C7
:1061E0002A71211D681D063E05F0B6FCB2B22A8157
:1061F000F02AE8D82800A11D0A3005F0ADFC0020E7
:10620000E2E7002310B50A789A4201D8900010BD49
:106210009A008A185488013304705488DBB2240A27
:106220004470948884709288120AC2700430EAE73D
:1062300010B51100029C062B04D004201022142B50
:1062400001D010BD022222714B7808781B02034353
:106250002380CB7888781B02034363800431601D60
:1062600005F07AFC0020ECE710B50C788B7804314F
:106270005C43E4B203702200013005F06DFC601C49
:1062800010BD0420022B06D10020537811781B0288
:10629000009A0B431380704710B50C000A88023136
:1062A00005F05AFC208810BD70B504000D0004985C
:1062B0001100012B01D8042070BD1678527812020B
:1062C000324302800200F83255701470E825002C29
:1062D00000D10C35023B9AB24280AA42EBD802317F
:1062E000043005F039FC0020E6E7042000998342E1
:1062F0000AD1537810781B0203430B80D37890782F
:106300001B02034300204B80704710B50C000A8825
:10631000023105F021FC208810BD000070B501217C
:106320001E000420049C0E400B4218D1CB40DDB26D
:106330008D4214D90A49DBB2098899420FD3230050
:10634000F6331D703300580011184978165C0902A5
:10635000314301332152D9B28D42F4D8002070BDAF
:10636000B844FF1F10B50C000A88023105F0F4FB99
:10637000208810BD10B50C788B7804315C43E4B2F2
:1063800003702200013005F0E7FB601C10BD10B562
:1063900011000298032B01D8042010BD1478527804
:1063A000043B120222430280CA788C7812022243F4
:1063B00042809AB28280F22AEED80431063005F08B
:1063C000CBFB0020E9E710B50C000B8803700B88AD
:1063D0001B0A43704B8883704B881B0AC3708A88E2
:1063E0000430063105F0B8FBA088043080B210BD3F
:1063F0000420012B03D100201378009A13707047FA
:1064000010B50C000B8803700B881B0A43704A8878
:106410000230043105F0A0FB6088023080B210BD6C
:10642000F0B589B003931E4B029242000700D05A88
:10643000019102F020F81325061E2DD0029B0124A5
:106440000370019B002B04D0001903999847001991
:1064500084B26B461B7A5BB2002B0FDA1021380036
:1064600002F01CFB1925002813D130003219E1B2CB
:1064700002F066FC051E0CD10C34A4B2042304AA5D
:10648000380005A993800696948101F0AFFD051EA2
:1064900002D0300005F0C8FB280009B0F0BDC046AE
:1064A0007466FF1F70B505000C0000280CD000209A
:1064B000814209D010222000044905F04DFB012043
:1064C0002B7823736B78637370BDC04650BF001187
:1064D000F0B506000D0017001C0085B002291BD086
:1064E0000020102907D1022B07D0102B03D115E073
:1064F0000020102C08D005B0F0BD69463800FFF729
:10650000D1FF2A0069460BE069463000FFF7CAFF59
:1065100022006946380004E0022BE9D12A00390044
:10652000300005F019F9E6E7031CF72800D9F72336
:10653000032008499AB2013A0B80D3170340064959
:106540009B189B100B80D30F04499B185B100B808A
:106550007047C046BC44FF1FBA44FF1FB844FF1F2A
:10656000034B1B888B4202D3024B4000C152704741
:10657000BC44FF1F7466FF1F014B4000185A704750
:106580007466FF1F1722014B1A8070477466FF1F45
:1065900070B505000E2005F09FF9041E13D0D0231E
:1065A000037000230622837007494570033005F00D
:1065B000D3FA064B2100DA8A62811B7E2373044BD7
:1065C000187805F0F1F870BD9066FF1F8066FF1F18
:1065D0000C45FF1F262803D8024B4000C05A7047C5
:1065E0000148FCE7BE44FF1FFFFF000070B5060036
:1065F0000C00094D1C220021280005F04DF9074B25
:106600001E70074B1C7005F017FB0123002801D0FA
:10661000002312202B7070BD8066FF1F0C45FF1FEA
:10662000A166FF1F70B505000D4C0800E260A16077
:1066300010220021656005F01FFB012803D1102105
:10664000A06802F058FD10220021280005F014FB7C
:10665000012803D11021606802F04DFD70BDC046D5
:106660008066FF1F70B5041E05D1002903D00622E5
:106670000D4805F071FA0D4B1D78012D11D1002C3C
:1066800005D102221A7005F04FFA280070BD0022D1
:106690001A70074B1B78FF2BF7D02000FFF778FF0D
:1066A000F3E70025F1E7C0469066FF1F8066FF1FF5
:1066B0000C45FF1F030010B5002801D1002010BDBC
:1066C00000780B4A002803D15988D1821B791376B0
:1066D0001378022BF2D10023984200D103331370B8
:1066E000044B1B78FF2B01D0FFF752FF0120E6E798
:1066F0008066FF1F0C45FF1F002911D000280CD019
:106700004B79012803D140225242134303E03F2238
:106710001340032802D001204B7170474022F4E758
:106720000800FAE770B5094D0100287800280BD061
:10673000074C0622200005F00FFA21002878FFF709
:10674000DBFF200005F080F970BDC046A066FF1F8A
:106750007A66FF1F00290AD0012808D13F224B7911
:106760009343C02B03D0403B5A425341981C70477F
:1067700070B5174D06002B78FF2B15D00A2005F0B9
:10678000ABF8041E10D0D0230370C83B8370114BAC
:1067900011491B784670C3700622043005F0DCF9FD
:1067A0002100287805F000F80C4B1B78012B0DD147
:1067B0000B4B1B68002B03D09B68002B00D0984725
:1067C000084B04211878084A05F0D6F870BDC04679
:1067D0000C45FF1FA066FF1F7A66FF1F9C66FF1F08
:1067E000C866FF1FCC66FF1F60EA0000014B986877
:1067F0007047C0468066FF1F014BDB681868704712
:106800008066FF1F074B10B5DA6813680133136009
:10681000054B1878FF2803D08021C90105F0BCF88A
:1068200010BDC0468066FF1F0C45FF1FF7B50E0068
:1068300002F0C8F8051E1CD00E4B06621F78002F10
:1068400000D10778AB791020019305F045F8041EBC
:106850000FD0D0230380C73B8370019BE91DC37019
:106860000622043005F078F921003800E66004F0D3
:106870009BFFF7BD0A45FF1F014B18787047C046C4
:10688000A066FF1F054B002805D1054B1A78054B64
:10689000002A00D1014B18007047C0469066FF1FC8
:1068A000A066FF1F7A66FF1F014B58687047C046FD
:1068B0008066FF1F024B1868431E9841C0B27047A4
:1068C000A466FF1F421E03000120152A03D9FF3BC7
:1068D0005A425341D8B27047F0B51C0000230E0055
:1068E00085B0039002920B70029A934201D300206C
:1068F00019E0E55C5A1CD2B2002DF8D0029851196B
:106900008142F4DC0233DFB2A35C18000193FFF78D
:10691000D9FF002807D0013D019A0399EBB23370EB
:106920008A4202D1E01905B0F0BDDB19DBB2DBE72A
:1069300010B50C0002F09EF803001220002B03D0CB
:106940002100588805F020F910BD000070B50E4DEB
:1069500084006359002B15D0186A002801D005F077
:106960003BF82B59586A002801D005F035F82B590F
:10697000986A002801D005F02FF8285905F02CF866
:1069800000232B5170BDC046B066FF1F1C4B70B575
:1069900004000E00150099420AD11A4B1B68002B07
:1069A00001D1122070BD1B68002BFAD09847F9E77F
:1069B000154B994215D1134B1B68002B0AD01B684D
:1069C000002B07D09847002804D1104B1C70104BA7
:1069D0001D70E7E729002000FFF7AAFF0028E1D19A
:1069E000F3E7080001F0EEFF0028DAD00378032077
:1069F000A342D7D12900300005F0C6F8D2E7C0463F
:106A0000FEFF0000AC66FF1FFFFF0000A966FF1F2E
:106A1000A866FF1FF7B50400808801F0D3FF0025AA
:106A2000A84203D00578A08802F008F81C4E3378FD
:106A3000002B1FD0AB421DD11A4B28001978FFF74D
:106A400077FF002818D000233370A3790820A77897
:106A5000A688019304F040FF011E0DD0D0230370DF
:106A6000CA3B8370019B477086808371280004F0C5
:106A70009BFE01E0002DE8D1A0880B4B8200D3588B
:106A8000002B01D0FFF762FF1721A088FFF768FDF8
:106A9000A08801F027FDA08801F0FEFDF7BDC046EB
:106AA000A966FF1FA866FF1FB066FF1FF0B587B07D
:106AB0001D000CAB1B88070001930DAB1B88142035
:106AC00002930EAB1B88160003930FAB1B8800913B
:106AD000049310AB1B88059304F0FEFE041E1AD02D
:106AE000D0230370CB3B47708370C6700622290009
:106AF0000430002D11D005F02FF8019B2100638197
:106B0000029B0098A381039BE381049B2382059B46
:106B1000A37404F049FE07B0F0BD04F0BDFEECE73D
:106B2000F7B5009308AB1B8807000C200D0016007A
:106B3000019304F0D1FE041E13D0280001F042FF9F
:106B400000280FD00078D0232370C93BA370009B8E
:106B500021002381019B6770A580E680638104F09A
:106B600023FEF7BD014B1878EDE7C0460C45FF1F2B
:106B700013B5040064890389C2888188C0780094B1
:106B8000FFF7CEFF13BD000010B5044C20680028AD
:106B900003D004F021FF0023236010BDB466FF1F63
:106BA000A122F0B5818892004A43384B384F1B68C8
:106BB00004009B189D2292009B18827989B01A606C
:106BC0003B68002B5FD01D78324B1B68002B04D034
:106BD0005B68002B01D00020984726000836310062
:106BE000E079FFF7B7FD237DE0710200E0780493C0
:106BF000638A29000393238A0293E3890193A3887C
:106C000000933300FFF752FFE378002B0BD1E289AA
:106C1000A379A18802920196E279280000920122CC
:106C200001F0DAFEE0703B68002B20D0FFF7ACFFEC
:106C3000194D287800281AD0184B1978FFF778FEDC
:106C4000002814D02B78E67808200793A78804F052
:106C500043FE011E09D0D0230370CA3B46708370E7
:106C600087808671079804F09FFD00232B70172101
:106C7000A088FFF775FCA08801F034FCA08801F023
:106C80000BFD09B0F0BD064B9DE7C0463409FF1F60
:106C9000B466FF1FC866FF1FA966FF1FA866FF1F17
:106CA0000C45FF1FF8B5070008000E0001F08AFE32
:106CB000041E18D02620FFF78DFC051E00D1257874
:106CC000062004F009FE041E0DD00021062204F067
:106CD000E3FDD0232370C23B21006770A370A68020
:106CE000E8B204F061FDF8BDF0B585B001930AABE0
:106CF0001B78070002930BAB1B7808000D00009275
:106D0000039301F05FFE061E22D0102004F0E4FD84
:106D1000041E1DD01022002104F0BEFD2620FFF726
:106D200059FC002800D13078D0232370C13BA370D8
:106D3000009B21002372019B67706372029BA580F8
:106D4000A372039BC0B2E3720C9BE36004F02CFDC2
:106D500005B0F0BDF7B50D00019001F033FE071E40
:106D600020D00E2004F0B8FD041E1BD02620FFF713
:106D700031FC061E00D13E78D0232380C53B06227D
:106D8000A370F91DE01C04F0E7FE019B2A0063815B
:106D90000123DD401A401D40210022736573F0B2CB
:106DA00004F002FDF7BD0000F0B585B002901000C0
:106DB0000D0017000A9E039301F004FE041E31D05B
:106DC000029B002B2ED1039B02795B0724D5122353
:106DD00013430422002E08D10B99002905D10C99E8
:106DE000002902D10D9900291AD01A430D9B227156
:106DF000002B00D0C9E0002E00D1CFE0002D00D044
:106E0000CCE0606A002801D004F0E6FD1C213000CF
:106E100004F03AFE606205E002239A430E33D7E79E
:106E200093432371654BBA00D458002C00D1AAE0DB
:106E3000002E10D0236A002B03D11C2004F064FE26
:106E400020625E4BBA00D358186A002803D01C2277
:106E5000310004F081FE0C9B002B12D0574CBB007C
:106E60001D596B6A002B03D1162004F04DFE686299
:106E7000BB00E358586A002803D016220C9904F08E
:106E80006BFE0D9B002B11D04C4DBC006659B36AB4
:106E9000002B03D1142004F037FEB0622B59986AFE
:106EA000002803D014220D9904F056FE380001F09A
:106EB00089FD051E67D0414BBA00D358002B62D024
:106EC0001A6A3420002A00D11C389A6A002A01D09C
:106ED000143080B20B9A002A01D01C3080B25B6A59
:106EE000002B01D0163080B204F0F6FC041E4AD00C
:106EF0001822002104F0D0FC2620FFF76BFB019044
:106F0000002801D12B780193D0232370029B20000D
:106F100063700A23294EA370039BBD00A371AB5974
:106F2000A780196A1830002905D01C22A06004F03F
:106F300013FE200034307359996A002907D00300EA
:106F400014221433E060029304F006FE02980B9BB7
:106F5000002B08D003001C221C330B9920610293E4
:106F600004F0FAFD02987359596A002903D01622D9
:106F7000606104F0F1FD6B462100187904F014FC07
:106F80003800FFF7E3FC05B0F0BD10220D9B0D9912
:106F90001B69A018236204F0DFFD2CE70B9B002B7C
:106FA00000D13FE7012D00D03CE7606A002801D006
:106FB00004F012FD1C210B982AE7C046B066FF1FA3
:106FC00010B5044C2068002803D004F005FD002310
:106FD000236010BDA466FF1F0B4B07B51A68002A7B
:106FE00001D100200EBD6946531C012012780731E3
:106FF000FFF772FC0028F4D002780123100018403B
:107000001A42EED0EEE7C046C066FF1FF0B51F4F34
:1070100001203B6887B0002B25D09B78059300F0BA
:10702000B3FB002821D00A20FFF7D4FA04000B207C
:10703000FFF7D0FA164B05001E78731E9E413B6881
:10704000F6B2191DD878FFF757FB3B682900DA7AAA
:10705000043303929A790193029200903300200046
:10706000059A04F0F1FD07B0F0BDFFF7B5FF002869
:1070700005D00620FFF7AEFA04000720D8E7082065
:10708000FFF7A8FA04000920D2E7C046A466FF1F54
:10709000A066FF1F70B50A4E040033780D00FF2B69
:1070A0000DD0042004F018FC011E08D0D02303707A
:1070B000CE3B45708370C470307804F075FB70BDB2
:1070C0001C45FF1F70B5040006200D0004F004FCF1
:1070D000011E0AD0D0230370CD3B8370054B447052
:1070E0001B688580187804F05FFB002C01D0FFF747
:1070F00067FF70BDA466FF1FF8B5264F06003B680A
:107100000D001124002B05D10522234B1B781342BF
:1071100002D112242000F8BD204A10241268002A4F
:10712000F8D01278002AF5D0DB0719D52B789A1EF3
:10713000012A1AD80C2004F0E7FC13243860002838
:10714000E8D000230A22437029000670023004F0C0
:1071500003FDFFF75BFF041E0AD0FFF731FFD9E7FD
:1071600000F012FB0028E1D1E4E7002BE2D0D0E7E9
:107170000B4B1B78032BCDD11D20FFF72BFA094BAE
:1071800018800028C6D0084B04211878074A04F05C
:10719000F3FBBFE7A466FF1FA166FF1FC066FF1FCA
:1071A000A066FF1F9E66FF1FCC66FF1F60EA0000FF
:1071B000F7B50193194B14001A78052306000F0048
:1071C00012201A4221D0012920D1154B1D68002D13
:1071D0001BD002201F2C18D8002C02D0019B002BA2
:1071E00013D0104B1F221E706E1C0021300004F0C3
:1071F00053FB01992200300004F0AEFC3100200066
:107200002C70002F06D004F097FAFEBD064B12201A
:107210001D68DCE704F0D8FBF7E7C046A166FF1F56
:10722000C066FF1F1C45FF1FBC66FF1FF8B50F4E51
:1072300012243368002B17D01B780F3C834213D1E4
:1072400000250B4F0221387804F04EFB094B042136
:1072500038781D8004F048FB074B28001D803368F8
:107260005C7004F029FC04002000F8BDA466FF1F38
:10727000CC66FF1FB866FF1F9E66FF1F70B5012812
:1072800023D11B4C2388002B03D01A4A1578002DDC
:1072900007D0194B1B68002B02D01878FFF7C6FFE8
:1072A00070BD3B2B02D93C3B2380F9E7134E0221F2
:1072B000307804F019FBFA222388920002215A4305
:1072C000307804F021FB2580EAE70B4B1B68002B8C
:1072D000E6D00B4B1B785B07E2D5084B02211878F0
:1072E00004F002FB0022024B1A80FFF769FED7E789
:1072F000B866FF1F9C66FF1FA466FF1FCC66FF1FBA
:10730000A166FF1FF8B51E4D2868002803D004F0C1
:1073100063FB00232B601B4E3068002803D004F071
:107320005BFB00233360184F05243B781800204096
:10733000234221D0154800F02BFA3B78234213D08A
:10734000202004F0E1FB2860002813D02022002137
:1073500004F0A2FA202004F0D7FB041E306005D010
:107360002022002104F098FA002004E0286804F0AC
:1073700033FB2C601320F8BD00F00AFAF4E7C04696
:10738000C066FF1FBC66FF1FA166FF1F1045FF1FE1
:1073900010B50A4C23681A1E0ED0002808D10130FF
:1073A000587004F089FB002805D02368002B02D018
:1073B0000021FFF787FE0122100010BDA466FF1F09
:1073C000F7B5274E050033680191181E21D05C786F
:1073D000244F012C30D1FFF7FFFD002825D02000DD
:1073E000FFF7F8F80400412814D91F4B0221187840
:1073F0001E4A04F0C1FA1E4B3C3C1C80022233683A
:107400005A703B78002B14D128000199FFF75AFEDF
:107410000120FEBDFA2292004243002AEED0124B18
:107420000221187804F070FAE8E7FFF7D3F80200B9
:10743000F3E700233B70EBE73B78002BE8D1032018
:1074400004F04AFA011E08D0D0230370CC3B4570EB
:1074500083703368187804F0A7F9FFF7B1FDD7E718
:10746000A466FF1F9C66FF1FCC66FF1F60EA00003A
:10747000B866FF1F10B51749838802008B4220D0E1
:1074800011D815498B4217D0144900205B1899B2C6
:10749000012907D8926811785A425341D8B2FFF7B0
:1074A000F9FD012010BD0E4A00209B1807229BB257
:1074B0009A424041C0B2F5E783681878FFF768FF49
:1074C000F0E7836899785A78090218781143FFF732
:1074D00077FFE7E70A20000006200000F8DFFFFF43
:1074E000AFDFFFFF014B18707047C0461D45FF1FFF
:1074F00010B5064C207001F041FA207804F04CFBE6
:107500000521207800F062FD10BDC046CC66FF1F4B
:107510000BB273B50D00002B00DBC4E0884B18786C
:1075200004F0C2FB041E0ED00378912B0FD0A22BC7
:1075300000D1A1E0834B1878FF2852D0210004F03D
:1075400033F900284DD180200002684076BD437891
:107550000F2B76D013D8052B70D00E2BEAD1808854
:10756000794B98422BD8794B98421BD8784B98424C
:10757000E0D1A3681878591CFFF774F838E03E2B67
:10758000D8D18378032B74D06CD8012B6ED0022B0A
:10759000D0D1704B1B68002B23D05B68002B20D010
:1075A00098471EE06C4BC0180C28C3D804F09CFA16
:1075B0001DC2C2150BC20B0B0B3223C23C00674B22
:1075C000C0180728B6D8664B1B68002B09D01B686B
:1075D000002B06D0200098470AE0A3681878FFF730
:1075E000C7F8200004F048FAADE7A068FFF762F89A
:1075F00000289FD0F5E7A3681B78002BF1D0554BEE
:107600001B68002BEDD01B68002BEAD021005548E9
:107610009847EDE74F4B1B68002BE2D01B68002B0F
:10762000DFD021005048F3E7504B1B68002BD8D027
:107630005B68002BD5D021004348E9E7FFF7EAF962
:10764000CFE780884A4B984203D04A4B984200D0FB
:1076500070E7464B1B68002BC3D05B68002BC0D083
:107660002100D5E7153B012BBBD963E7FFF798FA5B
:10767000B7E7FFF77DFAB4E73F4B1B78042B07D140
:1076800000236A4613800179408800F0C5FCA8E712
:10769000364B1B68002BA4D05B68002BA1D00100E7
:1076A000364898479DE7012421420AD0294B1B68A0
:1076B000002B04D05B68002B01D0002098470120EC
:1076C00043E78B070AD5264B1B68002B04D05B6869
:1076D000002B01D020009847022036E70421280023
:1076E00008400D4200D131E7254E3388002B21D0D0
:1076F000013B9BB23380002B1AD1FFF7DBF8002847
:107700000AD0204B1C70164B1B68002B04D05B6802
:10771000002B01D020009847FFF7C6F8694601F01A
:1077200001FD6846FEF7FEFF1D20FEF753FF308087
:1077300004200AE7024B187804F0D6F8F8E7C046B0
:10774000CC66FF1F1D45FF1F0E200000012000001A
:1077500009100000C466FF1FFEDFFFFFAFDFFFFF61
:10776000C866FF1F0C2000000B200000AC66FF1F46
:107770000D20000013200000A166FF1FFFFF000086
:107780009E66FF1F9C66FF1F10B501F09BF910BDA0
:10779000014B18607047C046C866FF1F0B88002069
:1077A000162B01D817230420014A13807047C046C6
:1077B0007666FF1F00207047074A03001188814248
:1077C00007D091880020994202D101308000101822
:1077D00070470020FAE7C046D466FF1FF0B58F78E7
:1077E00006000D00C7B01E2F15D1FFF7E5FF051EDF
:1077F00003D10024200047B0F0BD00223B0031003F
:10780000C078009200F0B2FB0400A81C00F0D3FB8B
:10781000FF23EB70EEE7264B062403931B78FF2B28
:10782000E8D0182FE6D87B08224A013BDB00029201
:107830009A589446002ADDD0029AD3185B68002B30
:10784000D8D00878002802D14B78012B02D1062429
:10785000122FCFD107AFAB88697800976446AA682A
:10786000A047041EC6D1AB78029A5B08013BDB003F
:10787000D318390030005B689847041E0BD1AB78F1
:10788000042BB6D0039A310010782200009700F044
:107890006DFB0400AEE76A78002AABD1AA7805A98F
:1078A0003B88087130000A704B80FEF747FBA0E769
:1078B0002045FF1F60BF00111D4B37B505009842E2
:1078C0000BD000290AD1FFF777FF002805D119480E
:1078D000FFF772FF002800D0058037BD01291AD1BB
:1078E000FFF76AFF041EF8D001235B420380A378F0
:1078F000FF2BF2D0FE2B07D00023E0781422009358
:1079000029001E3300F032FBA01C00F054FB0123C1
:107910005B426380E1E70229DFD1013901F0BEF863
:107920000028DAD12800FFF747FF041EDFD1D4E793
:10793000FEFF0000FFFF0000022210B5074B52427D
:107940001A80074801325A809A80DA8000F07EFA65
:10795000044801F025F8002010BDC046D466FF1F82
:10796000DD770011B97800110388F7B50400002B0A
:1079700002D102252800FEBD426802211378254865
:107980005268FEF7A5FD00282ED0234F01253A8826
:10799000002AEFD0802321885B0201259B1A99429F
:1079A000E8DC0C2004F0B0F8061E31D03B882288B9
:1079B0009C4600231800019561469DB2491989B281
:1079C000AA421BD8002801D062443A80002330002C
:1079D000082208C0210004F0BFF8104A1368002BE9
:1079E00013D100251660C5E76268022113780C48A0
:1079F0005268FEF76DFD0028C7D1BAE760681D0127
:107A00004019418101330198D6E71A001B68E6E767
:107A10001325AFE7CEBF00111E45FF1FD066FF1F25
:107A2000CCBF0011014B18707047C0462045FF1FA6
:107A300014230A0010B51A40194204D00122102163
:107A400001F048F810BD4B06F9D4012088434000EE
:107A5000F8E710B514008B0604D50122102101F0BF
:107A600039F810BD08230A001A40194202D14BB25E
:107A7000002B0FDA102101F02DF8002808D0230088
:107A8000F9331B78002BECD0F8342378012BE8D1A4
:107A90000020E6E703208907FAD4E2E7F0B51F00EB
:107AA000184B85B01C68019002910392002C27D1DD
:107AB000200005B0F0BDA5683301ED186B89019A6F
:107AC000934211D3029A93420ED8002F04D10A9BFD
:107AD000002B10D12C00EBE73B002978039A686853
:107AE000FEF7F6FC0028F2D10136B6B2A388B34205
:107AF000E1D82468DAE7A3680A9A5B891380E9E78A
:107B00000026F3E7D066FF1F37B50C000A884988C6
:107B10000123914217D3002A15D0651D23792A002D
:107B200002210A48FEF7D4FC102300280BD0237949
:107B30006188208800242A000094FFF7AFFF0A2301
:107B4000A04200D0230018003EBDC046CEBF0011A9
:107B500013B50A0008884988012388420BD80028F9
:107B600009D00024137905320094FFF797FF0A2308
:107B7000A04200D02300180016BD13B50A000888E3
:107B80004988012388420BD8002809D000241379A2
:107B900005320094FFF782FF0A23A04200D02300A1
:107BA000180016BDF0B58BB003904A8808880E0007
:107BB0000123824255D3002853D00023012704AC6F
:107BC00023700022718813000092FFF767FF051EE3
:107BD0003ED02078002835D12B78022B18D1677041
:107BE0006A8983000130E31880005A8069680222A4
:107BF000201803F0B1FF23780133DBB22370042B8C
:107C000019D93B006889013080B2002BD9D01FE020
:107C100002236370122358436A89231804305A8060
:107C200069681022201803F097FF23780133DBB234
:107C30002370002BE5D10C4A6B899B185A425341A3
:107C4000DBB2DFE76378012BE4D12B78022BC7D0BE
:107C500022780A23002A04D021000398FEF798F91D
:107C6000002318000BB0F0BD0100FFFF0F4BF0B573
:107C700004001868002816D083685D89A54207D8DB
:107C80008288AE18B44203DA12019A18934201D1E5
:107C90000068EFE71E005F891036A74204D1002973
:107CA00000D00D801800F0BD3300EFE7D066FF1F55
:107CB00070B505000C0008880021FFF7D7FF03000E
:107CC0000120002B04D022002800197AFFF7C1FE02
:107CD00070BDF7B50C00002501902300F6331B782A
:107CE000AB4201D800200AE06B00E65A00213000C8
:107CF000E718FFF7BBFF002802D126800130FEBD48
:107D0000017A0198FFF794FE002802D03B88238077
:107D1000F5E70135EDB2E0E710B504000888002171
:107D2000FFF7A4FF03000120002B03D02000197AE5
:107D3000FFF77EFE10BD0000054B1B68002B01D134
:107D4000180004E09A6852898242F6D198887047F8
:107D5000D066FF1FF0B50E27002687B0039302AB55
:107D6000FF183E8005001F4B40891400984207D041
:107D70002B78013000976A6880B2FFF78FFE06000B
:107D800002212B7818486A68FEF7A2FB00280FD062
:107D90006C892000FFF7D0FF002802D0013C0419B5
:107DA000A4B2039B002B00D01C80300007B0F0BDB4
:107DB00002212B780D486A68FEF78AFB0028E7D17C
:107DC00002212B780A486A68FEF782FB002807D058
:107DD000002EDED03B88A342DBD17489013CDFE773
:107DE0006C89DEE7FFFF0000CEBF0011CCBF0011A1
:107DF000CABF001110B50C00FFF7DEFC0300022023
:107E0000002B0AD0002C00D023609B781720FE2B7B
:107E100003D00138FF2B00D1002010BD73B50D0039
:107E200001A904001600FFF7E5FF172805D0002E72
:107E300004D129002000FEF727F976BD0122102188
:107E4000200000F047FE0028F3D0F6E7014B186051
:107E50007047C046E066FF1F37B56B469D1D0100A9
:107E600004000222280003F0DFFC2B88B02B0ED187
:107E70002379122B09D12300FF339B78012B06D1E4
:107E80000121608800F0E0F801E01B2BF8D037BD3D
:107E900010B5054B0421187000F098F8FFF74CFD61
:107EA000FEF770FB10BDC046E466FF1F0020F0B572
:107EB0000BB20F0087B0834234DA274B187803F0F7
:107EC000F3FE051E2BD00378A02B25D103AE310085
:107ED000FEF7E4F8041E0BD1B378DB0724D51F4B63
:107EE00006341B68002B03D03100688898470400D3
:107EF000A868002801D003F097FE002C08D1184A8A
:107F0000039B1340174A934206D0B3781B2B03D030
:107F10000121688800F098F8280003F0ADFD80206A
:107F20000002784007B0F0BD0F4B1B68002B10D04B
:107F3000310068889847041EDAD07378002BD7D1B7
:107F4000B27801A90A704B800C716888FDF7F6FFC2
:107F5000CEE70624F1E7C046E466FF1FDC66FF1F9C
:107F600000FFFF0000011200E066FF1FF7B501905F
:107F7000822040000D0017001E0003F0ADFC04003D
:107F80001320002C12D0B02320002370089BFC2269
:107F90006770658026710830002B08D0190003F047
:107FA000DBFD2100019803F0FFFB0020FEBD0899D6
:107FB00003F072FCF5E710B5041E06D00078FD282A
:107FC00003D803F061FCFF23237010BD0A1F93B296
:107FD00010B504000220032B05D882400020024B7C
:107FE000D1529B189C7010BD0467FF1F0B8870B5A1
:107FF000043B04000D000220032B0BD801212000BC
:1080000000F04CFD03001420002B03D029002000B9
:1080100000F0DEFB70BD000007B51300034A0092BC
:108020000A00012100F02CFC0EBDC0465582001153
:1080300007B5019203220092024B0A00122100F0C0
:1080400049FC0EBDD382001107B56B4601AA118011
:108050000449D88008780633012802D1190003F0BA
:1080600043FB07BDE566FF1F0C4B10B518700023DE
:10807000FF210B4A1380138193819380094A538017
:108080001370517293819372D174D38213755177A7
:1080900003F012FE00F0FCF910BDC0461467FF1F8C
:1080A0000467FF1FE666FF1FF0B58DB06B4600202A
:1080B00003910C229B5E834200DBB0E05D4B18789D
:1080C00003F0F2FD051E00D1A4E00378902B00D050
:1080D0009DE006AF01004688380000F013FA796889
:1080E0000400002900D19CE03B88052B6ED13B8920
:1080F000032B1CD905AC200000F0A2F86288172AD7
:1081000061D83989131D994231D1796823780431B6
:108110000291D90738D5607800F08EF9071E06D095
:10812000002303712378012B08D0132B23D0A868D8
:10813000002800D178E003F077FD75E062880299AD
:1081400009A800F0A6F80290380000F08BF909AAFF
:108150002378387A0192002231000092029A00F0CE
:1081600012F9380000F064F9029B002BDFD03000D8
:1081700000F080F9DBE70378032BD8D162880299FD
:1081800009A800F0D6F8DEE7122B13D1029909A84E
:1081900000F0B5F8021EEAD127498B88002BC6D023
:1081A000887909A92378019161780091310000F064
:1081B000EAF8BCE7002302AA93833000617809AA99
:1081C000FFF72AFFB3E71D4B0993F6E7042B02D014
:1081D0009A1F012AABD8184A043B9B00995A0029E0
:1081E000A5D0D218907831003A0000F0AEF80028FF
:1081F0009DD13B88042B03D001213000FFF724FFE1
:10820000012C04D1A868002801D003F00DFD28003E
:1082100003F032FC8020039B0002434018000DB0A5
:10822000F0BD012800D182E701213000FFF70CFFEB
:10823000EDE7C0461467FF1F0467FF1F010017002A
:108240000B7803704B784370CB788A781B0213430A
:10825000438070470A88030002700A88120A42703D
:108260000A88012A06D14A8882704A88120AC27096
:108270000420704702208242FBD14A8804309A7061
:108280004A88120ADA708A881A718A88120A5A7120
:10829000EFE710B50400012082420CD94B780A7830
:1082A0001B0213432380834206D1CB788A781B02BA
:1082B00013436380002010BD022BFBD1CB788A785A
:1082C0001B02134363804B790A791B021343A3807B
:1082D000F0E70B8803700B881B0A43704B88837090
:1082E0004B881B0AC3708B8803718B881B0A4371F0
:1082F000CB888371CB881B0AC371082070470300A9
:108300000120082A14D14A780878120202431A8000
:10831000CA788878120202435A804A790879120290
:1083200002439A80CA798879120202430020DA80D7
:10833000704710B504000120022A05D100204B78B7
:108340000A781B021343238010BDF8B506001020E5
:108350000F00150003F0C0FA04000120002C0ED01D
:10836000A0230C22290023806780201D002D07D028
:1083700003F0F2FB2100300003F016FA0020F8BDF4
:1083800003F08AFAF6E7F7B51E00009008AB142058
:1083900017001D78019103F09FFA041E12D0A2234A
:1083A0000370019B47704380099B057146710C2245
:1083B0000830002B07D0190003F0CEFB21000098F5
:1083C00003F0F2F9F7BD099903F066FAF6E737B55D
:1083D000041E0FD04388002B0CD00025C188132326
:1083E000007A172201950095FFF7CDFFFF236580E6
:1083F0006372257037BD000010B50C4904004A882F
:10840000002A09D08B89002B05D00020CB8A0222BC
:10841000834201D010BD012213000A2043430020F3
:108420004032C854C81842800472F3E7E666FF1F62
:108430000023438003707047094B00211A0010B5D8
:108440005C88002C06D01C79844203D10A234B435C
:10845000D01810BD01310A330329F1D10020F8E70B
:10846000E666FF1F10B50400407A03F00DFAFF2303
:10847000637210BD7047043010B580B203F074FA17
:10848000002803D00421494203F05EF910BD00002A
:1084900070B50025104CA0682580A581A580A84254
:1084A00002D003F0C1FBA56000250C4C0C4B606DA5
:1084B0001D80230058331D70A84202D003F0B4FB86
:1084C000656500256068002801D003F0ADFB01352B
:1084D00008340A2DF6D170BDAC67FF1F5067FF1F2F
:1084E000A067FF1F70B5041E09D1054D2880A88123
:1084F000A880A868002802D003F096FBAC6070BD8D
:10850000AC67FF1FF0B54B8885B001930023436033
:108510000A7905000F00022A00D07BE0CA88032AEE
:1085200017D98B685E7819783602DC78D8790E43D3
:1085300099781B7A24021B020C43034353495BBA0C
:108540000B80331D93421ED1042C04D0631F022BD9
:108550000ED9012015E0019A4D4B1201D35A002B80
:1085600006D00198FFF7BEFF4A4A13690133136131
:108570000421B8682E812C80494203F0E5F8686038
:10858000002005B0F0BD434D042C06D0631F022B24
:108590000FD9EB680133EB60DBE7019A3C4B12012A
:1085A000D35A002B05D00198FFF79CFF2B690133AC
:1085B0002B61374B30000293019B029A1B01019300
:1085C000002301998C468B52130063449C800393D3
:1085D0009E81FFF750FF039B041E986016D0042174
:1085E000B868494203F0B0F8FA880100043A200064
:1085F00003F0B2FA0199029AFB888A5A043B9B184D
:10860000029A8B522B6801332B60A2E7AB690133CE
:10861000AB619EE71E4B0293019B1E01029BF35A26
:10862000002B2DD002998C19A068002828D0012A8F
:1086300026D1FA889B189BB27352A189994217D30D
:108640009B1AC018B96803F087FA029BA289F35AF3
:10865000934200D07DE700222B81A3882B80A36862
:108660006B60029BF2520B4A53680133536070E710
:10867000084A9368013393600198FFF733FF68E776
:10868000044A536901335361F6E7C0461667FF1F7A
:10869000AC67FF1F1C67FF1F70B5051E15D10B4C83
:1086A0000B4B1880230058331870606D002802D0DF
:1086B00003F0BAFA6565250050356068002801D0DE
:1086C00003F0B2FA0834AC42F7D170BD5067FF1F17
:1086D000A067FF1FF0B51700A12285B0920001939B
:1086E0004243394B06001B680C009B18D933FF33FB
:1086F0001D78FDF741FF0430854204DD3000FDF7B1
:108700003BFF0430C5B2BD4207D33A000021300020
:10871000019B03F0A1FA05B0F0BD2900380003F079
:1087200073F92300C6B250331E700393019B2900D6
:108730006365380003F080F9CBB20293002B02D0BE
:10874000039B01361E7000262300503303931B78D1
:10875000B34204D8606D002831D10020DBE7029AD3
:108760002800002A04D0013B1000B34200D02800AA
:10877000F700E719387003F0A7FA786000280ED0E8
:108780003A78019903F0E8F9019A3B780136D31859
:108790000E4A0193D369F6B20133D361D4E7039B48
:1087A00018706065A74205D1084A1320D36A0133C7
:1087B000D362B0E7606803F037FA0834F2E703F0F9
:1087C00033FA00236365C8E73409FF1F1C67FF1FE6
:1087D000F7B50D0007000421686802F0B5FF2B898A
:1087E000040003702B891B0A43702B8883702B882D
:1087F0001B0AC3702E8902250436F6B2FB2E15D84B
:108800001B4B9F4214D10C2003F066F81135011E5A
:108810000CD0902303708E3B0371043B4380154BB7
:108820008460C680187802F0BFFF00252800FEBDD6
:108830005C237B43104AD3180093583301931B7871
:10884000002B0FD10300320038000099FFF742FFE0
:10885000019B05001B78002BE8D13800009903F03C
:1088600003F9E3E7054A0725536A01335362DDE75D
:10887000FEFF00001467FF1F5067FF1F1C67FF1FEC
:10888000F0B587B0009017200F0016000193FFF796
:10889000F2FD1325041E19D00C98031E02D0019975
:1088A000201D9847030AE370052302AAA070043034
:1088B000908127700098667003A993800494FFF755
:1088C00087FF051E02D0200003F0AEF9280007B094
:1088D000F0BD0000F0B587B01F000CAB1B78039112
:1088E000059301210DAB06001C78049200F0D6F828
:1088F0001425002821D02000FFF77EFD0135041E3D
:108900001BD01149059B0A7803700132D2B2131EA5
:10891000C68001D101231A000B7022713000049B24
:1089200003990097FFF7ACFF051E09D12300210032
:108930000648074A093302F0EFFF280007B0F0BDF0
:10894000002363802370F8E71867FF1FCF830011AF
:1089500030750000F8B505000E00064C064F236880
:10896000002B02D03100280098470434BC42F6D1D5
:10897000F8BDC046BC67FF1FD067FF1F0123064A32
:108980005B425380002313715362044A13605360A7
:108990009360D36013617047D067FF1FBC67FF1FF0
:1089A0000200002310B506499C000859002801D197
:1089B000625010BD0133052BF6D11320F9E7C046F4
:1089C000BC67FF1F034A5388181A4342584140426C
:1089D00010407047D067FF1FF0B585B002930AAB17
:1089E0001F780CAB1B88009008000E0001920393C7
:1089F000FFF7E8FF05001120002D1BD10E48FFF7FF
:108A0000E1FF04001520002C14D006220B99A77159
:108A1000E01D03F0A1F8019B30002371029B2900A7
:108A20006371009B66802370039B6562E381FFF79F
:108A300091FF280005B0F0BDFFFF000010B5FFF763
:108A4000C1FF04000220002C12D060880121FFF732
:108A500081FF606A002801D002F0BEFF28220021B9
:108A6000200002F019FF012300205B426380207187
:108A700010BD000030B5074A074C55880100137837
:108A80000020A54204D05B1A59424B415842104085
:108A900030BDC046D067FF1FFFFF0000084A10B579
:108AA00001230C00904208D0FFF78CFF031E04D076
:108AB000037923405A1E9341DBB2180010BDC04613
:108AC000FEFF0000024B1879431E9841C0B2704768
:108AD000D067FF1F70B504000D001600FFF772FF8E
:108AE000002804D10D4B9C4200D0143070BD416A67
:108AF00003790520002907D012221A40102A02D13A
:108B00000520002EF2D10F20DB06EFD5897E0C2048
:108B1000A9428941494249420840E7E7FEFF000077
:108B2000030010B5002800D110BD0348034A418856
:108B30009142F9D09847F7E7D067FF1FFFFF000089
:108B4000002330B5C45CCD5C6C40D4540133102B91
:108B5000F8D130BD0F23002210B5C45C640022435D
:108B6000CA54C25CD209013BF7D210BD0200010019
:108B700010B52032103102F0E7FE10BDF0B58BB019
:108B80000390102005931700049102F0BDFF0090A0
:108B9000102002F0B9FF009B13240190002B05D098
:108BA00000280CD11324009802F016FF019B002B23
:108BB00002D0180002F010FF20000BB0F0BD102012
:108BC00002F0A2FF0600102002F09EFF1324050011
:108BD000002E00D1AEE0002819D01022002102F0B2
:108BE0005BFE32002900039802F0AEFE041E0ED197
:108BF00033787F2B51D830000099FFF7ABFF009BF3
:108C00001B787F2B53D801990098FFF7A3FF300002
:108C100002F0E2FE002D02D0280002F0DDFE002C62
:108C2000C1D1102002F070FF0600102002F06CFF8E
:108C30000290002E7CD0002878D03A000F3223001A
:108C40000125121105D00F333B4015B25A42534152
:108C50001BB26A1E1201002B33D0049BD2B29818AB
:108C60000099029AFFF76CFF013D102200213000AD
:108C700002F012FEADB2049F2D017D19AF4242D029
:108C8000002C33D0300002F0A7FE029B002B00D155
:108C900089E7180002F0A0FE85E729003000FFF701
:108CA00059FF28002549009AFFF74AFFA7E7290046
:108CB0000098FFF74FFF28002049019AFFF740FF77
:108CC000A5E70F210F4004998A18D9B28F4208D91D
:108CD000D15C06A819540133102BF6D1029A0199E0
:108CE000C0E7791A48424141C901F2E73900300032
:108CF00006AAFFF725FF3200039806A902F024FE1A
:108D000010370400BAE7002CBCD13000029906AA43
:108D1000FFF716FF320006A9039802F015FE08229D
:108D200004003100059802F017FFABE71324A9E710
:108D30001324AAE7002800D06EE733E7D4BF001160
:108D4000F0B58BB00F0016000225009000283FD030
:108D5000002A3DD00B1DDBB21800029302F0D4FEB6
:108D60001135041E34D0FDF747FD05003A00009987
:108D7000201D02F099FEEBB20393E3702B0CDBB2E3
:108D80002F0A00936370FFB22B0E2370A77001931C
:108D9000FDF72CFD1022010006A802F085FE21003F
:108DA000029A04AB06A8FFF7E9FE051E0DD1039B4E
:108DB00008223370009B04A9B370019B7770F37095
:108DC000301D02F071FEFDF71DFD200002F004FED3
:108DD00028000BB0F0BDF0B58FB00D00149E0390CD
:108DE00004920593002A03D1022420000FB0F0BDA5
:108DF000002EF9D00398FFF7E5FD1424071EF4D0E8
:108E00007278337812021A43B3781B041343F27852
:108E100012061A43036A0192934201D30133E3D14C
:108E2000002D03D03B7901249B07DED508220021C9
:108E300006A802F031FD059B13240433DBB21800B1
:108E4000029302F061FE051ECFD0059A049904300A
:108E500002F02AFE04223100280002F025FE39002B
:108E6000102210310AA802F01FFE2900029A06AB58
:108E70000AA8FFF783FE041E0FD1082206A908A83E
:108E800002F012FE0822311D08A802F065FC01283C
:108E900007D101990398FDF7C9FC280002F09CFD59
:108EA000A3E70124F9E7000070B51C4C0500236816
:108EB000181E10D0002D14D11A78002A0CD1981C3D
:108EC000083202F049FE02F01FFF0135002808D1E8
:108ED00023681D70012070BD0A331800082202F0BB
:108EE0003BFE2368002BF5D0122002F0F5FC061E95
:108EF0000DD0C12321680370457002311022023069
:108F000002F02AFE23683100587802F04DFC2068F8
:108F100002F062FD00232360DCE7C046F867FF1F14
:108F2000F8B504002020FDF755FB0D4EA700BB59F6
:108F30000500002B0DD000280BD0D878FF2809D1D0
:108F400008492A000C55F35907480333611802F009
:108F5000E3FCF8BD290002F0E7FB0028F0D1F8E7B8
:108F60001468FF1FFC67FF1F79A1001170B5064D43
:108F700084006359002B05D0D87802F085FCFF22CD
:108F80006359DA7070BDC0461468FF1F70B50600E3
:108F90008CB00C00150000213022684602F07CFCE9
:108FA00031001022684602F07FFD1D2021000322BF
:108FB000684402F079FD6846FFF7D8FD2D210400D2
:108FC00003222800694402F06FFD20000CB070BD40
:108FD000F0B50700160097B001931CAB1D78302246
:108FE0001EAB00910AA800211C7802F055FC10224B
:108FF00039000AA802F058FD1022002102A802F050
:109000004BFC0722310002A802F04EFD072202AB02
:109010009818631E9C41019902F046FD02AB9C73B7
:109020002B005A1E934102AAD3730021102206A8D6
:1090300002F032FC06221D9907A802F035FD1A2025
:1090400002ABC01806221F9902F02EFD10220099D3
:109050000EA802F029FD102202AB0EA908781C7898
:10906000013A6040D2B2087001330131002AF5D1D3
:109070000AA8FFF77BFD102212A904000EA802F037
:109080006BFD102206AB0EA908781D78013A6840E6
:10909000D2B2087001330131002AF5D10AA8FFF7D6
:1090A00065FD044310222098E4B212A902F0FCFCF2
:1090B000200017B0F0BD70B50E0014008CB0010098
:1090C000102268461D0002F0EFFC3100082204A8BF
:1090D00002F0EAFC2100082206A802F0E5FC68463E
:1090E000FFF744FD04001022280008A902F0DCFC70
:1090F00020000CB070BDF8B506000D000024371933
:10910000AC4200D3F8BD02F03FFC030A3B70631C85
:10911000DBB201379D4203D90234F054E4B2EEE7EA
:109120001C00EDE773B506000C000225002819D0DD
:10913000002917D0032101A8FFF7DDFF6B469A79BC
:109140003F231A40013313436A463000937101A94B
:109150002200FFF71BFF051E04D10322E01C01A91A
:1091600002F0FAFC280076BD03785807DA08C00F31
:10917000D20080009B0710439B0F1843C0B270477A
:1091800007230B40C908C9000B4303707047000058
:1091900070B50400FFF7EAFE134DA4006359002BDD
:1091A00021D0186A002801D002F016FC2B59986EC5
:1091B000002801D002F010FC2B59D86E002801D0F5
:1091C00002F00AFC2B59186F002801D002F004FCB1
:1091D0002B59586F002801D002F0FEFB285902F0ED
:1091E000FBFB00232B5170BD1468FF1F0E4B80004A
:1091F000C35870B50C00002B0FD09D68002D0CD00B
:109200002B78201D0B706B784B70A97CFFF7B8FF93
:109210002B7E23726B69E36070BD10220021200059
:1092200002F03AFBF8E7C0461468FF1F014B1860D4
:109230007047C0461068FF1F074A0300800082582D
:1092400010B5002A06D0D088984203D1012901D157
:10925000FFF79EFF10BDC0461468FF1FF0B5264EF5
:1092600095B087000B93BB590500099112200A9213
:10927000002B31D0D888FFF7A5FB04001420002C68
:109280002AD0280010A9FFF7B1FFBB591E781D6A2C
:10929000002E23D00895FDF7EFFA07000020FDF718
:1092A000F1FA0790A379E61D069310AD0CA9089872
:1092B00000F0E2FA0EA9280000F0D7FA0B9B0A99F9
:1092C0000493069B09980293079B039601930097CA
:1092D0000EAB0CAAFFF77CFE15B0F0BDFDF7CCFA83
:1092E00006903000FDF7CEFAE31DA779079310AB87
:1092F00006000893DAE7C0461468FF1F30B50C4C2F
:1093000085002A59030085B00120002A0ED01800DC
:109310006946FFF76BFF2B591A78D888054B002A4E
:1093200000D1054B6A46072100F0D9FB05B030BDDE
:109330001468FF1F6B9800117998001130B5094C23
:109340008500295985B010226846253102F004FCB9
:109350002A591121044BD0886A4600F0C0FB05B0A1
:1093600030BDC0461468FF1F1599001130B5094C77
:109370008500295985B010226846353102F0ECFB92
:109380002A591121044BD0886A4600F0A8FB05B089
:1093900030BDC0461468FF1F53990011F7B54D4FFB
:1093A00086001020F4590D0002F0AEFBF359206244
:1093B000186A132200286CD0033A29009C6802F036
:1093C000CBFBF3591A780192002A58D11E6A227DEC
:1093D000317B944651400122019F114201D16746E1
:1093E0001740217D914339432175377B4F40BC465F
:1093F00060460027800701D44F0817400121022052
:109400008F40227D82433A432275377B5740BC46CA
:1094100060460027400701D497080F400420227DB2
:10942000BF0082433A432275627D0027944660461E
:10943000727B42400A4201D167460F400121627DA2
:109440008A433A436275777B5740BC4660460027A3
:10945000800701D457080F400220627D7F008243BD
:1094600017436775767B00227E40760701D4BA08E1
:109470000A400426617D9200B1430A4362756A780E
:10948000002A08D06278002A05D005220533DA7751
:1094900000221000FEBD04222979114205D1A17CD1
:1094A000114202D10533033AF1E7019A21782C7871
:1094B000002A02D10A002100140018220429E8D849
:1094C000042CE6D805206043034A05331218525C89
:1094D000DDE7C0461468FF1FE4BF001110B50A00A5
:1094E0001121024B00F0FBFA10BDC046AF990011EC
:1094F0000B0030B587B001AD2B806B460400110026
:10950000981D082202F028FB2A000B212000024BA4
:1095100000F0E5FA07B030BDD799001110B50A0088
:109520001121024B00F0DBFA10BDC0462B9A00114E
:1095300013B50B0011006A4613706B460400062237
:10954000581C02F009FB6A4608212000014B00F07C
:10955000C6FA13BD4B9A001110B50A001121024B37
:1095600000F0BDFA10BDC0469B9A00117FB5050002
:109570000B4BAA00D4580800002C0FD0666F237F35
:10958000E28821780396266F0296E66E0196A46E15
:109590000094FDF709FC2800FFF7FAFD7FBDC046E7
:1095A0001468FF1F10B51721FFF7E0FF10BD000082
:1095B00070B50A000D00064B0221040000F08FFA7E
:1095C000060029782000FFF7D1FF300070BDC046AB
:1095D0007B99001170B586B000236A4613708368CA
:1095E00004001D78681E0A2859D801A902F074FAEF
:1095F000060633373B3F43474B4F5300180000F0FC
:1096000042F9062312284BD000281BD16088FFF7AF
:10961000D9F90823002813D04279002A47D1264BD4
:109620001A78072312070BD5244B1A680723002A40
:1096300006D01668002E03D0290001AAB047030007
:109640006A4613706B461B786088002B2AD1FFF79F
:1096500067FC06B070BD180000F06CF9D4E7180084
:1096600000F087F9D0E7180000F093F9CCE7180074
:1096700000F0ADF9C8E7180000F0C3F9C4E718001E
:1096800000F0F6F9C0E7180000F0F6F9BCE71800A2
:1096900000F013FAB8E7180000F013FAB4E7072354
:1096A0006A46137069466088FFF782FFD1E7052399
:1096B000012AC5D1024BB8E7A166FF1F0C68FF1F46
:1096C0001068FF1FF8B52C4F8600F35904000D00F9
:1096D000002B40D0DA8882423DD15A78062A33D115
:1096E0001A78002A2ED0012099681A6A097D014251
:1096F00006D0157B054203D007225A700120F8BD21
:109700000220014204D0157B054201D00922F4E772
:109710000420014204D0127B024201D00B22ECE76C
:10972000164B1B68002BE9D05B68002BE6D02000AD
:109730009847BB5900215B78122BDFD12000FFF73F
:1097400015FFDBE70E4BECE7112A04D1002900D00E
:1097500032252900F2E7002D08D12000FFF732F969
:10976000002803D01023027913430371210028003D
:10977000FDF798FAC2E7C0461468FF1F0C68FF1F88
:109780001068FF1F70B50E4E8500AB590400002B0A
:1097900013D01B78002B11D10A4B1B68002B04D06F
:1097A0005B68002B01D02000984773595B78122B1F
:1097B00003D100212000FFF7D9FE70BD024BECE77A
:1097C0001468FF1F1068FF1F0C68FF1F094B800003
:1097D000C3581020002B0CD01A6A002A09D09B68AD
:1097E000002B06D0127A1B7E101C9A4200D9181C3E
:1097F000C0B270471468FF1F70B503000D0014005D
:109800000220002A30D000292ED013700B78081DBA
:1098100053704B789370FFF7A7FCE0700120022192
:109820002B7A23716B7B034063716A7B0A4013437D
:10983000042263716E7B1640334363716E7BF608BE
:10984000F600334363712B7B0340A371287B0140F7
:1098500000200B43A371297B0A401343A3712A7B89
:10986000D208D2001343A37170BD10B50A000100E5
:109870000120FFF7C1FF10BD10B50A000100022052
:10988000FFF7BAFF10BD70B506000C000220002ED5
:1098900030D000292ED07378201D0B70B3784B7018
:1098A000F178FFF76DFC01223579257271794B1043
:1098B000080013409340104003438810104080007C
:1098C000C9080343C9000B436373B1794B10080007
:1098D0001340934010400343881002409200C9088F
:1098E0001343C9000B4321202373FCF773FE854209
:1098F00001D2122070BD2220257AFCF76BFE854232
:10990000F7D823781820042BF4D86378012BF1D8EA
:109910000020EFE7030010B50220002909D0002B3A
:1099200007D00322481C0A7019000D3202F014F906
:10993000002010BD03000222080010B5002B06D045
:10994000002904D00E32591C02F006F90022100042
:1099500010BD030010B50220002909D0002B07D04C
:109960000422481C0A7019000C3202F0F5F800209D
:1099700010BD10B5FFF7DEFF10BD03000220002967
:1099800006D0002B04D0052200200A701B784B70F3
:10999000704703000220002B08D0002906D05B7816
:1099A00000200B70013B082B00D9183070470300D2
:1099B00010B50220002909D0002B07D00622481C30
:1099C0000A7019000A3202F0C7F8002010BD10B565
:1099D000FFF7B0FF10BD02000B00022010B50029F8
:1099E0000ED0002A0CD007211970118859701188E7
:1099F000090A997011180822D81C02F0ADF800204D
:109A000010BD03000A00022010B5002B0CD0002965
:109A10000AD099785878090201431180901CD91C0A
:109A2000082202F099F8002010BD030010B50220B2
:109A3000002909D0002B07D00822481C0A70190001
:109A4000921802F089F8002010BD02000B000220DD
:109A500010B500290BD0002A09D0092119701178FE
:109A600018185970511C062202F076F8002010BD1B
:109A700010B5FFF75FFF10BD02000B00022010B50C
:109A8000002A09D0002907D0517819701118062230
:109A9000581C02F061F8002010BD030010B5022030
:109AA000002909D0002B07D00A22481C0A7019008F
:109AB000063202F051F8002010BD10B5FFF73AFF52
:109AC00010BD02000B00022010B5002A06D00029AC
:109AD00004D018005178FFF753FB002010BDF0B5FB
:109AE00085B017001E006A46062305000800918114
:109AF0009380FEF7C0FC1324011E02900CD03800A6
:109B0000B047041E05D1280001A9FEF76FFA041E14
:109B100002D0029802F088F82800FFF701FA20002E
:109B200005B0F0BDF0B504008BB001911500002127
:109B3000102202A801F0B0FE334EA700B859002849
:109B40003CD0C388A34239D10378002B36D1427868
:109B5000062A18D102000100553235310C3006AB0F
:109B6000FFF7A9FA002829D12000FFF72FFE0200F5
:109B700006A902A801F0F0FF200002A901F024FECE
:109B800001200BB0F0BD816E002917D00B8A112A7D
:109B900028D19D420ED101981231093A01F0DCFD25
:109BA000012807D1BB5920009D6EFFF70FFE290049
:109BB0000200DEE732212000FFF7D8FC2000FEF78C
:109BC00001FF061E1BD0416A002918D00B8AAB4248
:109BD00015D108220198123101F0BEFD01280ED1E5
:109BE000716A0AE09D42E9D108220198123101F020
:109BF000B3FD0128E2D1BB59996E8A7EB9E72000F6
:109C000001F04AFDBCE7C0461468FF1FF0B56B4D7C
:109C100087007E5985B0337802900393002B00D0E3
:109C200087E0B368346A01937078062817D101225F
:109C30001B7D134202D0217B114218D10222134214
:109C400002D0217B114251D10422134203D0237B45
:109C5000134200D08BE0019B5A7DEB5991E007380D
:109C60000428F8D801F038FF032E42678300B36E52
:109C7000002B03D11C2001F047FFB066EB599C6E0E
:109C8000002C1CD010220021200001F005FE0298BB
:109C9000FFF79CFD01002000FFF72DFA01F074FE94
:109CA0002082200008211230FFF725FA0298FFF7E2
:109CB0008DFDA076EB592100D888FFF70FFC082214
:109CC000EB591CE0B36E002B05D01A00198AF088FE
:109CD0001232FFF70DFC0222019B197DEB59114254
:109CE0003DD0207B10423AD0073208E0F488FCF7E0
:109CF000DBFD01002000FFF711FC0A22EB595A702E
:109D0000029B9C002A595378073B042B11D8D0881A
:109D1000FEF758FE00284ED0C3895A08D2182849A9
:109D2000029B0298CB542B5941180433254801F06B
:109D3000F3FD05B0F0BDFCF79FFD03000120834259
:109D400001D100200393EB59DE88FCF79BFD0399BA
:109D500002003000FFF7ECFB019AEB59117D042261
:109D600011420CD0217B114209D00B22C7E7F688A3
:109D7000FCF73CFD01003000FFF7EEFB6BE7019ABA
:109D8000527D01210A4204D0607B084201D00C229E
:109D9000B5E702210A4204D0607B084201D00E22BE
:109DA000ADE704210A4204D0627B0A4201D01022AE
:109DB000A5E71222A3E7FA225200B0E71468FF1FBA
:109DC0001868FF1F83A1001110B5064B1A780423F1
:109DD000100018401A4200D00348FFF727FA00206D
:109DE00010BDC046A166FF1F2445FF1F70B50400CB
:109DF000FFF7D4FA051E43D12000FFF77FFA234E68
:109E0000A400A0598268937CDB0708D50321036A6C
:109E10001B790B40012B02D1017F0B430377431DBC
:109E2000D97F8B1E022B0DD8022900D00121C088BA
:109E3000FCF790FF042133591A7F59700A431A77AF
:109E4000280070BD01290CD102231022437000218B
:109E50000C3001F021FD305910213530FFF74BF95E
:109E6000EEE70529ECD10223D118437010220C3003
:109E700001F072FE04233259117F0B431377EAE796
:109E800008251828DCD1053DDAE7C0461468FF1F15
:109E9000F0B58BB0059143887E4F9E00F4591500B4
:109EA0000493002C15D1012902D000200BB0F0BD85
:109EB000101D57781678FFF757F9EB6832000293B8
:109EC0002B7A0499019300903B002000FCF70CFFD3
:109ED000EBE7E388049A934201D00820E6E7237871
:109EE000012B00D1D4E0059B581E092800D9CFE0F2
:109EF00001F0F2FD05CE0A29CC506C859AB22900FA
:109F00000498FFF773FFD1E72000290010224530A5
:109F100001F022FEB9594B78042B02D1013B4B7062
:109F2000C3E70B000A00253335320C310498FFF7E4
:109F300095F90498FFF702FA0522431E9841BB5990
:109F4000C0005A70B2E7200029001022553001F0FD
:109F500003FE049B4F4C9D00295904980A0006AB50
:109F600055320C31FFF77AF929591022453106A8EC
:109F700001F0F2FB012808D10498FFF7F7F90590EA
:109F8000002804D106222B595A7005988EE7082321
:109F90000593FAE763780C2B7AD1E36E002B03D19B
:109FA0001C2001F0B1FDE066BB59D86E00286FD0CF
:109FB0001022290001F0D0FDBB590498DC6EFFF798
:109FC00005FC0D22A076BB595A706EE7E06E0028A2
:109FD0005ED063780D2B5BD12B8808220382A91CED
:109FE000123001F0B9FDBB599A68517D022211422D
:109FF00026D0186A407B104222D00C32E4E7637806
:10A000000E2B45D1236F002B03D1162001F07CFDD0
:10A010002067BB59186F002803D01022290001F0D7
:10A020009BFD0F22BB59CFE763780F2B30D1206FF8
:10A030000622691C103001F08FFDBB599A68517DD2
:10A040000422114203D0196A497B1142D5D1002163
:10A050000498FFF78BFA28E7636F002B0DD0BB59EC
:10A06000586F0028F3D01022290001F075FD01225D
:10A07000BB5952425B6F1A61E9E7142001F044FDBD
:10A08000BB5960675B6F002BE9D126E72978DFE7D2
:10A0900007200BE71468FF1F10B5064C207001F075
:10A0A0008BFC06212078FDF791FF0348FEF778FC32
:10A0B00010BDC0462768FF1F3992001100200BB267
:10A0C00070B50D00834216DA264B187801F0ECFDCE
:10A0D000041E0DD00378922B0ED0A02B37D0224B2C
:10A0E0001878FF283AD0210001F05EFB002835D116
:10A0F00080200002684070BD43780E2B0BD03E2BB1
:10A10000EDD18378052B12D0082BE8D18179808896
:10A11000FFF7D8FA08E0154B82889A42DFD18368AE
:10A120001878591CFEF7C0FE002817D1D7E7104B4E
:10A130001B785B0712D50F4B1B68002B0ED09B685A
:10A14000002B0BD0C289811D80889847ECE7FFF770
:10A1500041FAA068002801D001F066FD200001F05E
:10A160008BFCC5E72768FF1F1D45FF1F1820000057
:10A17000A166FF1F1068FF1F10B50078FFF712FAE5
:10A1800010BD10B50078FFF7FDFA10BD0C23434356
:10A19000084A10B59B185A68002A03D0012901D13A
:10A1A000904710BD9B68002BFBD00029F9D1984740
:10A1B000F7E7C0464468FF1F01238340094A10B5F2
:10A1C000946B1C439463506B98435063D46B200092
:10A1D0009843012901D120001843D063116B0B4330
:10A1E000136310BD00800040F0B500240127154B1B
:10A1F00085B0DA6B144E03921A6C0192DA64019BFB
:10A20000E3403B4217D0039DE5403D400295E5B257
:10A2100002992800FFF7BAFF316A736A002908D053
:10A220003900002B01D0029979402800FFF7C4FFC4
:10A2300001E0002BF9D101340C36172CDFD105B029
:10A24000F0BDC046008000402868FF1F064B01217A
:10A250005A68C2400A4204D01B68C3401800084034
:10A2600070471B6DF9E7C046008000400122064B95
:10A270008240002903D0D9680A43DA607047D96860
:10A280009143D960FAE7C0460038004030B5032456
:10A2900044430F4BE25C1B199C785D7801232D1B16
:10A2A0000135AB40013BA340A140DB430C00122829
:10A2B00007D80849920052181168194021431160CB
:10A2C00030BD054A11680B4023431360F8E7C046D0
:10A2D0002BC0001108F0004014F00040C21F70B500
:10A2E000D4B20623092C0BD80125084C954000292F
:10A2F00008D00021FFF7CAFF23682B432360002307
:10A30000180070BD2368AB43F8E7C0460038004032
:10A31000214BF0B51B185B78022B21D10324444359
:10A320001E4A1F4EA35C1219947801221500854025
:10A33000B76B013CE4B23D43A240B563194C12280F
:10A3400015D89B0000290CD117495B1899680A435E
:10A350009A600123205C154A834011680B43136007
:10A36000F0BD11495B18996891439960F1E70E4B74
:10A3700000290DD159690A435A61225C1328E8D09B
:10A380000123203A93400A49086803430B60E7E73A
:10A39000596991435961F0E72868FF1F2BC00011EC
:10A3A0000080004070C0001100F00040A0F00040AC
:10A3B000A4F00040F8B500241B4E1C4D1C4B1B5D47
:10A3C000012B1FD1194A9269E2401A420BD0012297
:10A3D000B25693402200143AD2B2022A09D8154943
:10A3E0004A6913434B61013402360C35172CE5D111
:10A3F000F8BD0022B2560F499200521891680B43E3
:10A400009360F0E7022BEED1E7B23800FFF71EFFB2
:10A4100001235840C1B23800FFF77AFF3800FFF738
:10A4200015FF6877DFE7C046FDBF00112868FF1FF2
:10A430002968FF1F00F00040012202388240054BCE
:10A44000002903D059690A435A61704759699143F9
:10A450005961FAE700380040F8B50E0001210F00FD
:10A460008740114A0400D368FD43BB43D360831E79
:10A470008B4201D8FFF7E0FF00212000FFF72EFFFD
:10A480000A4A0B4B5168012E05D139431B19516003
:10A490005E700020F8BD2940516002221C196270D4
:10A4A0009A6915409D61F4E7003800400080004043
:10A4B0002868FF1F012210B58240074B002906D0F3
:10A4C00019680A431A600121FFF7C6FF10BD196819
:10A4D00091431960F7E7C046008000400C2370B537
:10A4E000002543430A4A29009B181D70094B0400AC
:10A4F0001B185D70FFF7B0FF0123A3400649280039
:10A500000A681A430A6005490A689A430A6070BDDE
:10A510004468FF1F2868FF1F3480004030800040DF
:10A5200070B504000E00FF2813D003250540FFF787
:10A53000D5FF084AA3089B009B183F22ED00AA40C4
:10A54000AE40196820009143314319600121FFF7A3
:10A550008DFE70BD18380040F8B50C244443134BF1
:10A560000500E4186368002B03D1A3681220002BB8
:10A570001AD0022201270E4B00215B195A702800C5
:10A580002770FFF769FF63681E1E08D0A3683E00AE
:10A59000002B04D02800FFF759FE4640F6B22800F1
:10A5A0003100FFF709FE0020F8BDC0464468FF1FD8
:10A5B0002868FF1FF7B5C420FF222B4B80001958D5
:10A5C000002491433F3A0A431A508022274F5202F7
:10A5D000274E1A60274B1D5D002D21D0A31E012B95
:10A5E00003D80121E0B2FFF727FF012D18D11F4B3F
:10A5F0009B69E3402B4213D0E3B218000193FFF7AD
:10A6000025FE01000198FFF755FFE3B2143B022B32
:10A610001DD801217156184A8D405369AB435361CF
:10A620003B7F002B0DD0E5B22800FFF795FF2800F7
:10A63000FFF70CFE7B7F0100834202D02800FFF76A
:10A64000A5FD01340C370236172CC3D1F7BD01210B
:10A6500000237156F3568D40074A9B009B189A6859
:10A66000AA439A60DCE7C04600E100E02868FF1FCB
:10A67000FDBF00112968FF1F00F0004010B5012147
:10A680000400FFF7E9FE0123044A002011194B7072
:10A69000A34091690B43936110BDC0462868FF1F1A
:10A6A00070B50E0015000400FFF718FF0C2363437C
:10A6B000094A20009B189D605E60FFF74DFFF02166
:10A6C000064B074A8900051E5A5002D02000FFF7AA
:10A6D00005FF280070BDC0464468FF1F0000FF1F33
:10A6E000E9A1001170B5134D07202C78002C1FD163
:10A6F000982221005200280001F076F90123C4209D
:10A70000FF222B700C4B80001C635C630B4B1C60A6
:10A710005C600B4B195891433F3A0A431A50802210
:10A7200052021A600D20074A074901F065F820001F
:10A7300070BDC0462868FF1F00800040A0F00040A8
:10A7400000E100E0B5A50011B5A30011030010B5AC
:10A750000620072B09D8054A137001F0CDFAD7213E
:10A760000020034B034A89005A5010BD4C45FF1F7F
:10A770000000FF1F151BFF1F70B51D0002240C29D0
:10A7800010D8094ACA40D2070CD5FBF72FFF041E88
:10A7900008D1059A04992800FBF744FFFCF7B2FDA5
:10A7A000FFF712FB200070BD1210000030B50D78CD
:10A7B00002232C009C43184201D02B431C00082587
:10A7C0002300AB43284201D02B00234320241D004B
:10A7D000A543204201D01C4325002A230D701842B6
:10A7E00004D011781E3B0B43137030BD0028FCD100
:10A7F0000C2113788B43F7E7F8B51D0006AB1B88D7
:10A80000140007AA0E000B201778002B27D10A7816
:10A81000022A49D14A68507811780002244A084334
:10A820008018042840D801F057F903121D1B23009B
:10A83000F06801F081F9021CC0B2B84200D93A1C9C
:10A84000D2B22000F1682A8001F086F906E00222E7
:10A85000F3681B882A8023701B0A63700020F8BDF0
:10A860000622EEE701232B80F3681B782370F5E7BF
:10A87000F368002B16D008222A801A8822701A88C2
:10A88000120A62705A88A2705A88120AE2709A8874
:10A8900022719A88120A6271DA88A271DB881B0A17
:10A8A000E371DBE72B80D9E701202B80D7E7C04697
:10A8B00000D6FFFFF7B516000A781D0008AB1F8809
:10A8C0000C000123022A18D14A685078117800023E
:10A8D0002B4A0843801803280FD801F0FDF8022501
:10A8E0004439E06801F028F9C0B20723B84204D324
:10A8F0007B190193152B02DD0D231800FEBDE068C6
:10A900002A003100C01901F027F96B4600209B880E
:10A91000E268D0541B4B1B68834203D01B68834200
:10A9200000D098470023E8E70B23002FE5D1022D44
:10A93000E2D1737832781B021343E2681380114B23
:10A940001B68002BEED01B68002BEBD00120E8E742
:10A950000B23002FD1D1062DCED12A003100E06883
:10A9600001F0FAF8DEE70B23002FC6D1012DC3D189
:10A9700032787533012AC0D8E3681A70D2E7C0462E
:10A9800000D6FFFF346AFF1F70B50C0015000728C2
:10A9900037D801F0A1F8041436361B36242E1820BF
:10A9A00015290BD8184E16220021300000F074FF34
:10A9B00022002900300001F0CFF8002070BD1820DF
:10A9C0000229FBD11288114B1A80F6E718200829BA
:10A9D000F4D10A000E48290000F026FFEDE7182008
:10A9E0000129EBD10B4B10780B49DA69FFF7DEFE3A
:10A9F000E3E718200129E1D1064B10780749DA6B0B
:10AA0000F4E70220DAE7C0461C6AFF1FCA45FF1FB1
:10AA1000C045FF1F5045FF1F7845FF1F9845FF1F8A
:10AA2000030010B50020DB0704D50721024A0348C4
:10AA300000F08CF810BDC04688C000115045FF1FC3
:10AA4000054A03001068002803D082889A4201D189
:10AA5000806870470068F6E7386CFF1F0A880300BB
:10AA600008009A4204D08A8804309A4200D000201C
:10AA700070470000F8B5F82200230D4F0D4E79689D
:10AA8000050042433370994200D07B600A4C00219C
:10AA9000200000F001FF00231A007C60AB4202D1CD
:10AAA00000203370F8BD01332280DBB2F834F5E7C3
:10AAB000386DFF1F346DFF1F3C6CFF1F73B56B4675
:10AAC00001900600684615001980FCF74DFF041E32
:10AAD00011D1002D0FD07689002E11D00C2001F05D
:10AAE00013F800280ED0084A046013688680856039
:10AAF000002B02D11060200076BD1A001B68F7E71A
:10AB00000224F8E71324F6E7386CFF1F0121002226
:10AB10000A4B10B549420A4C198099809A719A7073
:10AB2000084B2070012019805A60FFF7A3FF20789E
:10AB3000FCF778FF0448FDF733FF10BD3C6AFF1FA8
:10AB4000406DFF1F386DFF1FF9AB0011022310B5D8
:10AB5000002802D0FFF7B2FF0300180010BD00006C
:10AB6000030010B50020DB0704D50421024A034886
:10AB7000FFF7A4FF10BDC0469CC00011D045FF1FC9
:10AB8000F0B50E2687B003930CAB1F8802ABF61806
:10AB90000500080031000292FDF768F8040001206A
:10ABA000002C0FD03088FFF74BFF03000E20002B46
:10ABB00008D05E68002E05D021002800039B029A71
:10ABC0000097B04707B0F0BD0A4B10B5984207D1C7
:10ABD0000122002352420A808B708A808B7110BD43
:10ABE000FFF73CFF0028FAD001235B4203800023DB
:10ABF0008370F4E7FFFF0000F8B5050001290AD1D2
:10AC0000134E00243388F827AB4219D0280011498D
:10AC1000FFF7DAFF06E0022904D10139FDF73EFF14
:10AC20000028EDD0F8BD3B0063437268D018D35ABA
:10AC3000002B09D03A00002100F02EFE0134E4B2CE
:10AC4000054B1B78A342EED801235B423380DDE73E
:10AC5000386DFF1F3C6AFF1F346DFF1F10B5FFF7F3
:10AC6000FDFE03000020834200D0987810BD000054
:10AC7000F0B589B01C000EAB80CB03901E8810ABE2
:10AC80001B78049202930B7A0D00DB0616D42B7806
:10AC90000593022B24D00498FFF7D2FE002812D08F
:10ACA00003689C46002B0ED0029B220001932900D2
:10ACB0003B00644603980096A04705E00498FFF720
:10ACC000BFFE002802D10E2009B0F0BD8368002B22
:10ACD000F9D00A222900039898470028D7D0F3E733
:10ACE0006B6858781A786B4B000210439842D2D8A0
:10ACF000043B984210D2684B984242D015D8674B1B
:10AD0000C0180128C7D80B20002EDDD1EB681A78B7
:10AD100059683A80200028E0614BC018032800D908
:10AD200079E000F0D9FE846A789E5E4B9842B2D1F9
:10AD30000B20002EC8D101233B80EB6831001B782B
:10AD400023706889013080B2FCF790FF3A88031EB7
:10AD50000ED0017802328A183A80428962704289A4
:10AD6000120AA27059680278E01C00F0F5FE06E0B5
:10AD700004323A8031000422601C00F08DFD002076
:10AD8000A2E70B20002E9FD1EB6807A91E880423A1
:10AD90003B80330A300026706370FCF767FF051EA6
:10ADA00028D004AB9A890E2304A95B183E49C668D3
:10ADB000FCF7D0FF00280BD12B783C486A68059936
:10ADC000FBF786FB002803D1012304AA5B42D38151
:10ADD0003278022A06D17168201D00F0BDFE3B8842
:10ADE00002333B800E2304AA9B181B88A3701B0A06
:10ADF000E370C4E704ABDE81F4E70B20002E00D043
:10AE000062E7E9680398FFF729FF02233B8020707F
:10AE1000000A6070B3E70B20002E00D054E7022236
:10AE2000EB681B883A8023701B0A6370A7E7E86809
:10AE300000F082FEC2B203000720B24200D243E714
:10AE40000DD00299DBB27118994202DB921BD3B28A
:10AE50000293029BE9681A003B8089195AE7002394
:10AE6000F6E70B20002E00D02EE70722EB683A8091
:10AE70001A7822705A7862705A88A2705A88120A18
:10AE8000E2701A792271DA886271DB881B0AA37179
:10AE900075E7C046042900000228000000D8FFFF23
:10AEA000FFD6FFFF03280000FFFF0000CCBF00110A
:10AEB000F0B58DB06B460020089120229B5E834246
:10AEC0003DDAA64B187800F0EFFE071E32D003786B
:10AED000B02B2CD10079023816281FD800F0C4FC02
:10AEE00017001E001E001E0031001E0096001E00EE
:10AEF0001D011E0052011E0073011E00CD011E0027
:10AF000050021E001E001E008E021E00E302944B23
:10AF100094491B8878880B80FBF71AF83800FCF7F7
:10AF20009BFF914B1B68002B01D0380098473800DD
:10AF300000F0A2FD8020089B0002434018000DB0E5
:10AF4000F0BDF6220021874800F0A6FC0BAA3B7B4F
:10AF50007989388900923A000D32FCF79FFD040090
:10AF6000804B1B78002C3FD146E0804B78880593BE
:10AF70007F4B4100CB5A0BAE073BDBB232880293CA
:10AF8000002301937B4B210006930093059BFFF761
:10AF90006FFE744D002810D1069B3A8A1B889A4296
:10AFA0000BD138000599123000F0D6FB002804D0F0
:10AFB0002B7862899B00EB185A80162306A81B1871
:10AFC000328820007989FCF7C5FE2B7804009A00AE
:10AFD000AA1851880029C3D00133DBB22B70002896
:10AFE00007D006A9C98A9180634A12889A42BCD8C0
:10AFF00002E0012149429180002B04D05949788810
:10B00000FAF7DAFF8AE73E890A2479E000253E89CB
:10B01000574B06937B88069A5B009B5A033B9D42E5
:10B0200002DB002DF0D05BE0162206A812183B7B55
:10B03000798900923A0030000D32FCF72FFD05901F
:10B04000002858D04689017A7888FCF7F1FC041E64
:10B0500044D1464B78880793069B4100C95A454B1B
:10B060000439C9B206AAD28A0693029101940093C8
:10B070000599079BFFF7FCFD041E2FD1069B39495C
:10B080001A88931C002D26D14B807988384B4900B3
:10B09000CB5A5119033B8B4220DD059B31485B891C
:10B0A00041190B71A91C0135C9B2EDB205914519C1
:10B0B0001B0A2B71059B2D490433181800F04CFD19
:10B0C0002C4B059A1B88D318DDB22C4B9E4205D021
:10B0D0000136B6B29CE749889942D6D0002D0CD0F3
:10B0E000204C2800618800F027FE2070210078881D
:10B0F000FAF772FF12E7059CF0E7002C00D183E716
:10B100007B78142B00D109E716493B794E800B70F0
:10B110000C717888FAF712FF00E7162406ABE418E2
:10B1200021003889FCF7A2FD011E00D1B7E1788823
:10B1300022880F4C45002C5B0A4D013CE4B202947E
:10B1400000240F4B01940095FFF792FD041E00D0E0
:10B1500014E129007888FAF74FFFDFE6406DFF1F02
:10B16000BC44FF1F446AFF1F386AFF1F3E6BFF1F6E
:10B170007466FF1F346CFF1FBA44FF1FFFFF0000FF
:10B18000466AFF1F162406ABE41821003889FCF735
:10B190006DFD011E00D182E178882288AE4C450009
:10B1A0002C5BAE4D013CE4B202947C89AC4B019423
:10B1B0000095FFF75DFD041E00D0DFE029007888D0
:10B1C000FAF724FFAAE60025A44B1D803B00FE33BE
:10B1D0001B78A24A78880792AB4208D99E4B128806
:10B1E0000693069943005B5A013B9A4203DB079999
:10B1F000FAF716FF92E616246B00FB18059306ABD0
:10B20000E418059B21001889FCF730FD011E03D1CD
:10B21000059B01241E8973E77888924B2288069C3F
:10B22000099343001B5B904E013BDBB2029300236A
:10B2300000960193099BFFF71BFD041E02D0059B9E
:10B240001E895DE77B88069A5B009B5A079A1088E7
:10B2500032881218934202DC1B1A013B33807F4C68
:10B26000023032880999001900F076FC2388328870
:10B2700001359B182380EDB2A8E70BAA3B7B7989A7
:10B28000388900923A000D32FCF708FC0025059041
:10B29000059B002B04D10A24002D00D16EE060E054
:10B2A000059B7888197AFCF7C3FB0100041E63D163
:10B2B000694C6C4B788806940993069B4400E45AC9
:10B2C000694B063CE4B20BAE3288079302940191BD
:10B2D00000930599099BFFF7CBFC041E4CD1079BFB
:10B2E0005E491B881A1D002D30D14A80059B5B4C9E
:10B2F0005A8963191A716B1C9BB2E318120A1A71EE
:10B30000162306A832881B1879890598FCF722FDB8
:10B31000FF21AA1C2E1D03350B00059092B2B6B278
:10B32000ADB2002803D006ABDB8AD9B21B0AA21843
:10B33000651911712B714C4D301D2A88494920180F
:10B3400000F00AFC2B88F618B5B2A1E749889142B3
:10B3500007D17A8806995200525AEB18053A9A4258
:10B36000C4DC3E4C2800618800F04EFB20702100B8
:10B370007888FAF75FFED1E5002DF2D13E89BFE66D
:10B38000162606ABF61831003889FCF76FFC3D0035
:10B390000400FF3500282DD0037A9B060CD4002230
:10B3A0007B893989788800923A000C32FFF7E8FBF4
:10B3B000041E10D03E8915E03088FFF741FB0028BD
:10B3C0001AD08368002B17D0210012227888984762
:10B3D000041EE4D0EEE7AB78002B02D17888FAF7B0
:10B3E00039FE0026AB78002B00D097E5002C00D169
:10B3F00094E585E60124DDE70E24DBE7162506ABA0
:10B40000ED1829003889FCF731FC041E47D0037A77
:10B410009B0611D4154A7B881188994203D01448A1
:10B42000814207D11380134BF8261D780023D9B22F
:10B43000A94221D30924A1E72888FFF701FB0028AE
:10B440002FD08368002B2CD02100122278889847B7
:10B45000041EDFD092E7C0467466FF1F446AFF1FD8
:10B46000466AFF1F3E6BFF1F346CFF1F386DFF1FC6
:10B47000FFFF0000346DFF1F310059435468013352
:10B480006018615A0029D2D13C0008342100F8220A
:10B4900000F062FB21007888FAF7E4FD3EE5012424
:10B4A0006CE70E246AE71D4B1A887B889A4231D0DC
:10B4B0007888FAF7E1FD31E5F823059851684343B0
:10B4C000CD18C95A00291FD03B7A012B0BD16C88AB
:10B4D000AB887888AA1D0094FFF752FB041E02D0A7
:10B4E00000233B722E88F8220021280000F0D4F9B6
:10B4F00000232B80059B0133DBB20593084B059994
:10B500001B78064A8B42D7D801235B421380002C5C
:10B51000CED0F5E5002634000596EFE7386DFF1F25
:10B52000346DFF1F70B504000E001500FFF796FA8A
:10B53000031E08D131000548FFF790FA03001120DF
:10B54000002B02D01C8000209D7070BDFFFF00000A
:10B55000F8B50B4F06003B780D001400FF2B0ED002
:10B560000A2000F0B9F9011E09D0B123038000239D
:10B5700046800371C5800481387800F015F9F8BD64
:10B580001146FF1FF7B50F0008A90600088809A992
:10B590000B240988002821D10234022B1ED15578B2
:10B5A00013782D021D432B008B4301937334002B22
:10B5B00014D1FB68300019000093FFF74FFB019C8A
:10B5C00085420BD02A0030000099FFF7ABFF041E24
:10B5D00004D12A0030007989FFF7BAFF2000FEBDB0
:10B5E000F0B50E7885B003900AA805880120022ED8
:10B5F0000DD14C682778647824023C43054FBC4247
:10B6000005D10398DBB201960095FFF7BBFF05B0AB
:10B61000F0BDC0460229000010B504000C4800F03F
:10B62000E3F80C48A16B00F0DFF80B48E16B00F089
:10B63000DBF80A48216C00F0D7F8094B0948196873
:10B6400000F0D2F8084B1B68002B00D09847FEE7AB
:10B650007EBE001194BE0011A3BE0011B2BE001147
:10B6600004ED00E0C1BE0011446DFF1F002307B5CB
:10B6700001A80193FFF7D0FF044A0548002110B547
:10B68000121A00F009F9F8F79BF9FEE7486DFF1F61
:10B690001446FF1F0000000001B40248844601BCAC
:10B6A000604700BF091B000001B40248844601BC8A
:10B6B000604700BF8D34FF1F01B40248844601BCBF
:10B6C000604700BF4D32FF1F01B40248844601BCF1
:10B6D000604700BF2526000001B40248844601BC33
:10B6E000604700BFA532FF1F01B40248844601BC79
:10B6F000604700BFE117000001B40248844601BC66
:10B70000604700BFA54F010001B40248844601BC58
:10B71000604700BF056A000001B40248844601BCCE
:10B72000604700BF350E000001B40248844601BCEA
:10B73000604700BF5147010001B40248844601BC84
:10B74000604700BF4D1F000001B40248844601BCA1
:10B75000604700BF5549010001B40248844601BC5E
:10B76000604700BFCD4C010001B40248844601BCD3
:10B77000604700BFE139FF1F01B40248844601BCA5
:10B78000604700BFCD34FF1F01B40248844601BCAE
:10B79000604700BF3555000001B40248844601BC33
:10B7A000604700BF6DBC000001B40248844601BC84
:10B7B000604700BF594F010001B40248844601BCF4
:10B7C000604700BFA137FF1F01B40248844601BC97
:10B7D000604700BF311B000001B40248844601BC31
:10B7E000604700BFC56D010001B40248844601BC3A
:10B7F000604700BFE53A010001B40248844601BC3D
:10B80000604700BFED32FF1F01B40248844601BC0F
:10B81000604700BFED4A010001B40248844601BC04
:10B82000604700BF0189000001B40248844601BCA2
:10B83000604700BF810E000001B40248844601BC8D
:10B84000604700BFC9A9000001B40248844601BC9A
:10B85000604700BFB14E000001B40248844601BCFD
:10B86000604700BFF539FF1F01B40248844601BCA0
:10B87000604700BFE53CFF1F01B40248844601BC9D
:10B88000604700BF6D3AFF1F01B40248844601BC07
:10B89000604700BF1147010001B40248844601BC63
:10B8A000604700BF154D010001B40248844601BC49
:10B8B000604700BF3D18000001B40248844601BC47
:10B8C000604700BF7530FF1F01B40248844601BCC9
:10B8D000604700BF055E000001B40248844601BC19
:10B8E000604700BF1D4D010001B40248844601BC01
:10B8F000604700BFB352010001B40248844601BC56
:10B90000604700BF1D36FF1F01B40248844601BCDA
:10B91000604700BF8B52010001B40248844601BC5D
:10B92000604700BFA946010001B40248844601BC3B
:10B93000604700BF2146010001B40248844601BCB3
:10B94000604700BF156B010001B40248844601BC8A
:10B95000604700BFE548000001B40248844601BCCE
:10B96000604700BF0124000001B40248844601BCC6
:10B97000604700BFE928000001B40248844601BCCA
:10B98000604700BF5952010001B40248844601BC1F
:10B99000604700BF2951010001B40248844601BC40
:10B9A000604700BF0D52010001B40248844601BC4B
:10B9B000604700BF6532FF1F01B40248844601BCE6
:10B9C000604700BFC926000001B40248844601BC9C
:10B9D000604700BF5522000001B40248844601BC04
:10B9E000604700BF014C010001B40248844601BC1D
:10B9F000604700BFB70E000001B40248844601BC96
:10BA0000604700BFADAE000001B40248844601BCEF
:10BA1000604700BF090E000001B40248844601BC23
:10BA2000604700BFC51D000001B40248844601BC48
:10BA3000604700BFC94A010001B40248844601BC06
:10BA4000604700BF090E000001B40248844601BCF3
:10BA5000604700BFC521000001B40248844601BC14
:10BA6000604700BF9DA9000001B40248844601BCA4
:10BA7000604700BF7D18FF1F01B40248844601BC27
:10BA8000604700BF434D010001B40248844601BC39
:10BA9000604700BFF94C010001B40248844601BC74
:10BAA000604700BF2D35FF1F01B40248844601BC2A
:10BAB000604700BF4551010001B40248844601BC03
:10BAC000604700BF691F000001B40248844601BC02
:10BAD000604700BF6571010001B40248844601BCA3
:10BAE000604700BFD13CFF1F01B40248844601BC3F
:10BAF000604700BFBD3CFF1F01B40248844601BC43
:10BB0000604700BF193BFF1F01B40248844601BCD7
:10BB1000604700BF3D4B010001B40248844601BCB0
:10BB2000604700BF2539FF1F01B40248844601BCAD
:10BB3000604700BF291C000001B40248844601BCD4
:10BB4000604700BFDD52010001B40248844601BCD9
:10BB5000604700BF4550000001B40248844601BC64
:10BB6000604700BFE94C010001B40248844601BCB3
:10BB7000604700BF2D3AFF1F01B40248844601BC54
:10BB8000604700BF8552010001B40248844601BCF1
:10BB9000604700BF8D12000001B40248844601BC1A
:10BBA000604700BF5D17000001B40248844601BC35
:10BBB000604700BFB54C010001B40248844601BC97
:10BBC000604700BFC130FF1F01B40248844601BC7A
:10BBD000604700BF7138FF1F01B40248844601BCB2
:10BBE000604700BFC53F000001B40248844601BC65
:10BBF000604700BF456B010001B40248844601BCA8
:10BC0000604700BFC13BFF1F01B40248844601BC2E
:10BC1000604700BF2124000001B40248844601BCF3
:10BC2000604700BF7D37FF1F01B40248844601BC56
:10BC3000604700BFD949010001B40248844601BCF5
:10BC4000604700BF5125000001B40248844601BC92
:10BC5000604700BF851F000001B40248844601BC54
:10BC6000604700BF5118FF1F01B40248844601BC61
:10BC7000604700BFAD3AFF1F01B40248844601BCD3
:10BC8000604700BF1D4B010001B40248844601BC5F
:10BC9000604700BF75A9000001B40248844601BC9A
:10BCA000604700BFF30E000001B40248844601BCA7
:10BCB000604700BFF54E010001B40248844601BC54
:10BCC000604700BF7918000001B40248844601BCF7
:10BCD000604700BF017F000001B40248844601BCF8
:10BCE000604700BFEDA5000001B40248844601BCD6
:10BCF000604700BFDD66010001B40248844601BC14
:10BD0000604700BF151BFF1F01B40248844601BCF9
:10BD1000604700BFD91B000001B40248844601BC43
:10BD2000604700BFC95C010001B40248844601BC01
:10BD3000604700BF953BFF1F01B40248844601BC29
:08BD4000604700BF350E000052
:10BD480000020103020203030403050206020702BC
:10BD5800080209030A030B030C020D000E030F036C
:10BD68001003110313031403150016009D3D001161
:10BD7800D13D001100000000020000008ABD001142
:10BD8800192A0F180A000000F1590000FD240000CC
:10BD980041460100A9800011BDA0001111750011D4
:10BDA800AD7E001191530011B1AE0011F94F001191
:10BDB800953F0011C5400011000000001616000054
:10BDC80002000000D4BD0011F4FFF3FFD2FC000014
:10BDD8000542001100000000000000005475796160
:10BDE8000042312E33003030313400676974687591
:10BDF800622E636F6D2F7076767800544830350068
:10BE0800020000001CBE0011292A282A272A262AF7
:10BE1800252A242A0A180000E20400007102000002
:10BE280078EC0000744000001027000060F000006B
:10BE380006640000204E000000000000050000001D
:10BE48001F501D00023CB400000115001300000043
:10BE5800A1020000303132333435363738394142A7
:10BE680043444546005048592B36325858504C5593
:10BE78005330353034005B48617264206661756CFC
:10BE8800742068616E646C65725D0A004C522020F3
:10BE9800203D203078253038780A00504320202073
:10BEA8003D203078253038780A0050535220203D04
:10BEB800203078253038780A0049435352203D20F5
:10BEC8003078253038780A0095570011E957001165
:10BED8000000000002000000E8BE00116F2A6E2A70
:10BEE8001A18EAD8BC80F0FC6000000000000000CE
:10BEF8000000F303B59747D6F613F7D777E6F0A710
:10BF0800F474000001A00000000000006410B71DD8
:10BF1800C8206E3BAC30D9269041DC76F4516B6B6F
:10BF28005861B24D3C7105502083B8ED44930FF031
:10BF3800E8A3D6D68CB361CBB0C2649BD4D2D386E7
:10BF480078E20AA01CF2BDBDFB349B5F8000008034
:10BF58000010000000000000136100119D7700111F
:10BF680037610011A57B0011BB6100117B7B0011BB
:10BF780031620011517B001183620011197D00119B
:10BF8800EB620011197D00111D630011D37C0011B3
:10BF980031620011097B0011A9620011B17C001106
:10BFA80000000000000000008F630011B17C001148
:10BFB800F1630011B5770011052A042A012A002A25
:10BFC8000229032801280028011800180000000091
:10BFD80000000000000000000000008701010201CD
:10BFE800020101020102030304010301010101012D
:10BFF8000303020103000D000E00100011001300DE
:10C008001401070108010A010B011C011D020402A9
:10C0180005020702080219021A021C021D03010385
:10C02800020317000201000504000807000B0A00BC
:10C038001716001D1C010201010504010E0D011156
:10C0480010011413011716011A19020201020B0A32
:10C05800020E0D0211100214130217160305040331
:10C068000807030B0A030E0D0001020307090A0B58
:10C078000E0F101112141718191A1B1F2021220055
:10C08800F9A70011B5A80011000000000200000087
:10C09800D2BF001100000000E1B50011000000004F
:08C0A80002000000D0BF0011EE
:020000041FFFDC
:1000000000000000F93E001190BD00118CBD0011F0
:100010002063FF1F0000000000000000000000003F
:1000200000000000000000000000000000000000D0
:1000300000000000000000000000000000000000C0
:1000400000000000000000000000000000000000B0
:1000500000000000000000000000000000000000A0
:100060000000000000000000000000000000000090
:100070000000000000000000000000000000000080
:100080000000000000000000000000000000000070
:100090000000000000000000000000000000000060
:1000A0000000000000000000000000000000000050
:1000B0000000000000000000000000000000000040
:1000C0000000000000000000000000000000000030
:1000D0000000000000000000000000000000000020
:1000E0000000000000000000000000000000000010
:1000F0000000000000000000000000000000000000
:1001000000000000000000000000000000000000EF
:1001100000000000000000000000000000000000DF
:1001200000000000000000000000000000000000CF
:1001300000000000000000000000000000000000BF
:1001400000000000000000000000000000000000AF
:10015000000000000000000000000000000000009F
:10016000000000000000000000000000000000008F
:10017000000000000000000000000000000000007F
:10018000000000000000000000000000000000006F
:10019000F134FF1F3933FF1FC1660100000000006A
:1001A000000000000000000000000000000000004F
:1001B000000000000000000000000000000000003F
:1001C000000000000000000000000000000000002F
:1001D000000000000000000000000000000000001F
:1001E000000000000000000000000000000000000F
:1001F00000000000000000000000000000000000FF
:1002000000000000000000000000000000000000EE
:1002100000000000000000000000000000000000DE
:1002200000000000000000000000000000000000CE
:1002300000000000000000000000000000000000BE
:1002400000000000000000000000000000000000AE
:10025000000000000000000000000000000000009E
:10026000000000000000000000000000000000008E
:10027000000000000000000000000000000000007E
:10028000000000000000000000000000000000006E
:10029000000000000000000000000000000000005E
:1002A000000000000000000000000000000000004E
:1002B000000000000000000000000000000000003E
:1002C000000000000000000000000000000000002E
:1002D000000000000000000000000000000000001E
:1002E000000000000000000000000000000000000E
:1002F00000000000000000000000000000000000FE
:1003000000000000000000000000000000000000ED
:1003100000000000000000000000000000000000DD
:1003200000000000000000000000000000000000CD
:1003300000000000000000000000000000000000BD
:1003400000000000000000000000000000000000AD
:10035000000000000000000000000000000000009D
:10036000000000000000000000000000000000008D
:100370006DB6001100000000000000000000000049
:10038000000000000000000000000000000000006D
:10039000000000000000000000000000000000005D
:1003A000000000000000000000000000951AFF1F80
:1003B000000000000000000000000000000000003D
:1003C000000000000000000000000000000000002D
:1003D000000000000000000000000000000000001D
:1003E000000000000000000000000000000000000D
:1003F00000000000000000000000000000000000FD
:081838005071FF1F4118FF1F52
:10184000024981F3088802F02FFC00005071FF1F4D
:1018500010B502F081FA072804D0122808D0022817
:1018600008D010BD044A0420136B01331363F8E75A
:101870000220F6E71420F4E71C67FF1FF8B5070005
:101880000C0026002500503630785135002804D150
:101890000300287058342370F8BD2978CA00481E08
:1018A0008141A3183800A25C5B68C9B2FFF7D0FF82
:1018B00000280DD12B78DA00A218013350602B706C
:1018C0003378044A013B3370136A01331362D8E75B
:1018D0000123DFE71C67FF1F5C234343074910B563
:1018E000C9180B0058331B78012B05D1FFF7C6FF31
:1018F000034A936A0133936210BDC0465067FF1FCD
:101900001C67FF1F10B502F0A7FB064A0121130058
:1019100010CB4942D967044B136002F08DFC2000C4
:1019200010BDC04600E100E01000100010B504003A
:1019300002F092FB024B1C6002F07EFC10BDC04620
:1019400000E100E010B5040002F086FB4021094AE6
:10195000200013688B43136002F0FEFB01F0AAFD28
:101960000022054B01201A60044B04321A6002F079
:10197000D3FBFEE71CF00040C4F00040C0F0004084
:10198000431E5A425341A022F0B5D2015B4213409C
:10199000154D164A40019B182A18127E8BB00191F2
:1019A000002A1BD01A000832D46F0022E6B206AF1C
:1019B000E4B294420EDC2818C369002B08D00199C8
:1019C00002AA117106AA049202AA167303A89847E4
:1019D0000BB0F0BD1978B9540132EAE71A7D1A78D4
:1019E00006AB01261A70E6E7DC69FF1F00400040E5
:1019F000F0B5254B04004001C25C85B0002A2BD015
:101A00001A18117E002927D0917E002924D011793F
:101A1000022921D11689D788D168F51BADB22A1CBD
:101A2000102D00D9102292B2BE4217D118180123EE
:101A300003710023C269C38003819A4206D06846BD
:101A4000032103730171029301A890470820002C21
:101A500000D0192001F026FC05B0F0BD013C654224
:101A60006C41A0256442ED012C40084D1B186419FF
:101A7000074D0633013A92B2AA42EDD01888461CAF
:101A80001E80085C2070F5E7DC69FF1F0040004005
:101A9000FFFF00000F220E4B10B59868104002386F
:101AA0000A280BD802F014F90D0A0B0A0A110A0AC7
:101AB0000A0A060002210020FFF762FF10BD012183
:101AC000F9E70020FFF794FFF8E7DB6FF6E7C04681
:101AD000004000400F220E4B10B5986810400238AD
:101AE0000A280BD802F0F4F80E0A0B0A0A120A0AA6
:101AF0000A0A060002210120FFF742FF10BD012162
:101B00000800F9E70120FFF773FFF7E7DB6FF5E760
:101B10000090004013B5334C2378072B3DD8324B4F
:101B20001A78324B002A39D18022196852020A43AE
:101B30001A60252001F07AFF20232D4A11680B43FB
:101B4000802113606B460422C905086807331042E0
:101B500028D080210422C905C86810422ED08021D7
:101B60002020C905CA688243CA6014221A701A78F4
:101B7000002A2FD18021C905C86820320243CA60DB
:101B800014221A701A78002A28D11A4B1A7D22784A
:101B90005A601D221A705932DA6013BD1A6816494C
:101BA0000A40C5E7086802430A6014221A701A78CE
:101BB000002ACED01A78013AD2B2F7E7C8680243B9
:101BC000CA6014221A7019784A1ED2B21A700029FB
:101BD000F9D1C4E71A78013AD2B2C7E71A78013AC4
:101BE000D2B2CEE74C45FF1F1446FF1F3CF0004029
:101BF0004445FF1F00200040FFFFFEFF564B70B51D
:101C00001B68012B03D1554A936D0133936502F094
:101C10009BFA534B534A1860534B544C1A600123A0
:101C2000534A1360534A13602378002B06D00622D0
:101C30005149524802F098F900232370504A514B01
:101C400010681B78C1B2002B0ED14F4CC0B2237864
:101C50005BB2002B4FDB237824785BB264B21B04A9
:101C600024021B191B1813600B1C50294ED950233A
:101C7000464A47491078DBB2FF2202284BD1086858
:101C8000444C454D267890432A78964254D9227880
:101C900024782E78023B5D10A31B6B435201D31AAC
:101CA00010335B111843086002F04EF9031F012B3B
:101CB00045D83A4B1B78002B06D0394B1B78002BAC
:101CC00002D0002002F0F8F9A122364B9200997858
:101CD000354B4A431B689B18832292009B181B7844
:101CE000033B012B03D8AF20400002F0A5F80122EE
:101CF0002E4BDA8270BD237824785BB264B2FF3356
:101D0000FF341B0424021B190138ABE7CAB2022AB4
:101D1000AED20223ACE70868254C264D26789043C6
:101D20002A78964208D9227824782D78023B5B10D5
:101D3000641B63435201B2E72378DBB2B2E70228A7
:101D4000D5D11D4B1B78013B022B03D91B4B1B78B4
:101D5000022BCCD16C20C8E79809FF1FFC0FFF1F96
:101D60005466FF1FFF3F0000141003405866FF1F1A
:101D70000C10034000100340D50BFF1F7211FF1F12
:101D8000B40003408C09FF1F680AFF1F490AFF1FA8
:101D900094000340460AFF1F470AFF1FF908FF1F70
:101DA0002209FF1F300DFF1F3409FF1FBC0BFF1F4F
:101DB000440AFF1F450AFF1F1C09FF1F2309FF1FBD
:101DC00010B502F0E9F90022014B1A8010BDC0469F
:101DD0005066FF1F10B502F007F9A121054A8900DE
:101DE0009478054A61431268044B5218528C1A8049
:101DF00010BDC046300DFF1F3409FF1F5066FF1F86
:101E000010B50D4B0D4A9978A1239B004B431268E6
:101E1000D218531DD97F0A4B1B88994209D2441C02
:101E200007D0C82805D0D2695B1A5A43054B5343E3
:101E3000C01802F0E9F910BD300DFF1F3409FF1F73
:101E40005066FF1F7102000070B5244D2B68002BF7
:101E500028D002F0C9F92B68D8402B680400002B69
:101E600027D002F031F92B68D8401D4B1D4A9978D4
:101E7000A1239B004B431268D118D25C91239B0095
:101E8000002A20D0CA580132CA50174B17491B6884
:101E90000868834214D3D23B181A012A1AD0144B73
:101EA000186070BD02F0A0F9124B196802F024F816
:101EB000D3E702F009F90F4B196802F01DF8D4E7D7
:101EC0000D495B18E8E7CA500C4B1B68DB68E41847
:101ED000201AE4E7F530FF30E1E7C0461C08FF1F99
:101EE000300DFF1F3409FF1F9C09FF1F5466FF1FA1
:101EF000A009FF1F1808FF1F2DFF3F005C66FF1F92
:101F000070B504000D00282916D10300A433C2883F
:101F10001B889B1A0B4A9BB293420DD906006A3666
:101F200005223100653001F0EFFE002804D13100B8
:101F3000200002F051F970BD2900200001F0B4FF2B
:101F4000F9E7C046FE7F0000F8B50400012002F06A
:101F50007BF802F0E9F80300184A19491060886A12
:101F60008D6AA842FBD1174D174E28607568AC46A4
:101F7000164D2F680025BC4501D275687D1B144E97
:101F800000193560C862A4204C6A400320434862AF
:101F900010490978002905D00F490978022902D192
:101FA0000F3B1360F8BD012901D1083BF9E7032974
:101FB00001D1053BF5E7033BF3E7C046E408FF1F0B
:101FC00000F00040340AFF1F28100040180AFF1FCD
:101FD0001C0AFF1F1C09FF1F4A0AFF1F70B580243F
:101FE0001025E405A3682B43A36001F0F5FEA36868
:101FF000AB43A36070BD0000F7B5160080221C0043
:102000001023D2050191916805000B4393600022D3
:102010005A4BD7301A6001F0F7FF9D232A002F009A
:102020009B00EB58CA3201210092FC37002B01D0F3
:102030000021009A386802F067F82900009BCB3134
:102040001A784F4BD3351A604B780A781B0213432A
:102050008A7812041A43CB781B061343494A1BBAE9
:1020600013604B790A791B0213438A7912041A43CD
:10207000CB7931001B061343434A1BBA13606B78BC
:102080002A781B021343AA7812041A43EB781B0622
:1020900013433E4A1BBA1360019A330213433C4A6E
:1020A00013603C4B22001B1B9C4603293DDCB308FC
:1020B0009A0013005142B21A032A46D1354AE01859
:1020C000511A82784078120400020243E05C043323
:1020D00002430A600022FF2B4BDDF0222E4B12013F
:1020E0001A600F222D4B1A602D4A1368002BFCD06A
:1020F0000023224A27491360091B321D0B191B6854
:10210000043A180A23706070180C1B0EA070E3705C
:102110000434002AF2DC802210213B68D20501330E
:102120003B6093688B439360F7BD6346D5789818FE
:1021300093782D061B042B43157804392B435578CF
:1021400004322D022B430360AFE7022A0AD1114A61
:10215000E05C511AE2185278120202430A6004331A
:102160009BB2B7E7012AB5D10A4A521AE15C116065
:10217000F5E7084959180A600433ACE70000044049
:102180003C00044038000440340004403000044067
:102190000C0004400001044004000440100004400E
:1021A00014000440F7B5150080221C001023D2054E
:1021B0000091916807000B4393600023654AD73074
:1021C000136001F021FF9D233E009B00F9583B0066
:1021D000CA363200FC33002900D07FE0586801F095
:1021E00093FF390032785C4BCB311A604B780A7818
:1021F0001B0213438A78AC4612041A43CB78281D7D
:102200001B061343554A1BBA13604B790A791B020C
:1022100013438A7912041A43CB791B061343504A9D
:102220001BBA13604B7A0A7A1B0213438A7A120490
:102230001A43CB7A21001B0613434A4A1BBA136088
:10224000009A2B021343484A13602200474B1B1B82
:102250000093009BCE785B1801938B7836061B04A5
:1022600033430E78043833434E7804313602334317
:10227000019E33600328ECDC0321A808431C9B006B
:102280002940800003292BD13849E5185E18A97828
:102290006D78E35C09042D02294319433160030082
:1022A00008330021FF2B2DDD314B324919600F21FE
:1022B000314B1960012327490B60304B1968002905
:1022C000FCD006211B680B40042B20D0802200206C
:1022D000D20593680A318B439360FEBD01217DE7EF
:1022E000022908D121495D18E1184978E35C090207
:1022F00019432960D3E70129D3D11C495918E35C5C
:102300000B60CCE71948181801600433CAE70023B2
:1023100010490B606346002B0CDC3B00FC335A6811
:10232000102101325A608022D205936801208B432C
:102330009360D2E7009B9B181B68190A13705170B9
:10234000190C1B0ED37004235B4291709C44043221
:10235000E0E7C046000004403C0004403800044070
:1023600034000440300004400C00044000010440EC
:1023700004000440080F0000100004401400044052
:1023800070B5061E19D00222614B9B799343012B35
:1023900013D1604B1A78FF2A0FD15A78FF2A0CD13B
:1023A0009A78FF2A09D1DA78FF2A06D11A79FF2A0A
:1023B00003D15B79FF2B00D1A7E0574B0C201A7893
:1023C000012A08D00022554D1A702B781A00093ABC
:1023D000042A01D8212070BD5A1F012AFAD94C4C79
:1023E000A07B042800D990E0A279032A00D98CE0D0
:1023F000821E012A03D862881F2A00D885E0002E99
:1024000061D0012E00D080E0A288012AE2D0002B0A
:102410000AD10138032803D801F05AFC151D1915FB
:102420001F202E7001F088FD2B785A1E032A16D823
:1024300000253B4B1D602823237501F02DFDA8428C
:102440002ED0A580C6E7022320202B70EAE70423C4
:1024500022202B70E6E7032321202B70E2E7073BC5
:10246000012BB7D82F4B1B68DB6A9B06B2D52E4BCE
:102470001A78002AAED1A27B911E012901D9002A27
:10248000A8D1022280211A702823284D890128789A
:10249000237501F091FC80212878890101F0ACFEC0
:1024A0000123A380224B1B78002B0AD0FA22802123
:1024B000204B92001B8809025A431C4B187801F0EC
:1024C0003BFC002087E701F0C7FD2B78A680073B87
:1024D000012B06D918482E7001F03EFD1E2001F098
:1024E0002BFD114B114C1A78002A06D080210022B6
:1024F000207889011A7001F05FFC01F09DFE8021B7
:102500002078090201F058FCDBE7122063E7C0469F
:10251000A60BFF1F6B09FF1F1A09FF1F1C09FF1FD6
:102520004809FF1F5C66FF1F2309FF1F1B09FF1FD0
:102530002109FF1F2C09FF1F0010004010B50029C2
:1025400001D001F079FD10BDF7B5604B019199788C
:10255000A1239B004B435E4A060014681022E41836
:10256000D6235B00E0583623FF33E35C0027934318
:10257000222B41D1574B0F3A1A600760012501F019
:102580004BFE019B1880E8235B00E35C002B01D02D
:10259000B34258DD0023504FFB70AD33FF33E35897
:1025A0001A68002A03D09B88DB439B071DD0382381
:1025B000FF33E35C002B18D09B235B00E35C002B14
:1025C00013D1D133FF33E35CB3420EDAA4235B00B3
:1025D000E15AE018090A023101F01EFD2300012230
:1025E000FE33013E01351A87FA70E8235B00E35C95
:1025F000002B2AD0A8B2FEBD03683D00002BBED040
:1026000081880430090A023101F006FDD6235B00FF
:10261000E3581F60B2E72300B133BA00FF33985884
:10262000013781880430090A023101F0F5FCE82302
:102630005B00E35CBB42EEDCE822F61AED180023F7
:102640005200A354A6E70027F1E7200001F094FD13
:1026500000281FD0002E1DDD73198826471901930D
:10266000B600200001F0D8FB5A30800020184068E6
:10267000013581880430090A023101F0CDFC2000C7
:1026800001F0F2FCA3590133A351BD4202D0019BDA
:102690009D42E6D1114BE35C002BABD095239B0010
:1026A000E35C002BA6D00E4BE15A0029A2D00D4AC4
:1026B000A35C994202D90133A3549BE700231A215A
:1026C0002000A35401F030FB94E7C046300DFF1FFB
:1026D0003409FF1F00140340E010FF1F5A020000DE
:1026E000720200005E020000F8B51D4B1D4F1A7803
:1026F000002A10D1BA7B002A02D101321A7003E0FD
:10270000032AFAD0022AF8D001F0C6FB00220120E9
:10271000154B1A70F8BD154B154D1C68154B9E785E
:1027200001232B702878C0B200F0CEFCBB7B002BBD
:102730000BD101F0A1FCA1239B007343E418832378
:102740009B00E41823782B70E4E7032B02D101F0FF
:102750006BFCF0E70020022BDCD101F0C5FBEAE7BF
:102760001C09FF1FA60BFF1F2309FF1F3409FF1FB2
:10277000490AFF1F300DFF1FF0B587B00EAD2F784F
:102780000FAD2D780593AC46634614000E4D0CAA90
:1027900012782E7803930D9B009201932200059BE3
:1027A000029701F071FB2E70012C01D0042C08D18E
:1027B000802206498B889343054A1278D20113433D
:1027C0008B8007B0F0BDC0461C09FF1F6C11FF1FB6
:1027D0007809FF1F0B001B3B70B504003020E02B75
:1027E0000DD81300E025493BFF3B9BB2ED00AB4207
:1027F00005D8034B200019825A8201F03DFB70BDC1
:102800008410FF1F10B501F09FFC054B00205B6892
:10281000052B04D9034A5268D20200D4980810BD8F
:1028200000100040FCE100E070B501F015FC0D4B1C
:102830001B68FC33DC691D6AFFF7E4FF64198442FE
:1028400004D2094B01241B68002B07D0042200246A
:10285000064B1A70064A93690133936101F0ECFC50
:10286000200070BD5C66FF1F9809FF1F2309FF1F32
:10287000FC0FFF1F70B50C4D2B68FC335C6A01F038
:10288000EBFBFFF7BFFF2B680025FC339B6AE318C7
:10289000834204D2054B1B68AB4200D1051B01F0FB
:1028A000CBFC280070BDC0465C66FF1F9809FF1F67
:1028B000D722044B92009B5810B5002B00D09847AC
:1028C00010BDC0460000FF1FF0B587B001F08AF9C7
:1028D000FFF7EEFFC54BC64C04931B78022B45D186
:1028E000C44B1B68186A01F0AFFBC34BC34A1A60A4
:1028F000C34BC44A1A60A022C34B52001A60049B07
:10290000187801F0E9FAC149C14801F0E5FBC14975
:10291000C14801F0E1FB1022C04BFF201A60802269
:1029200052031A60802292031A60802212041A60F5
:1029300001F0C2FB012001F007FAFA20400001F08B
:102940004BFB582001F078FAB54801F01DFA012040
:1029500001F082FA072001F0CFFBE26DB14B1A4083
:1029600084235B001343E36507B0F0BD01F01CFB5B
:10297000AD4E0290322001F067FB33681B0628D46D
:102980003C2001F061FB0F2001F05EFB974B1B78B0
:10299000012B00D113E1802533682B4200D0A1E048
:1029A000636C03202B43636401F04EFB01F0FCFADF
:1029B000029B0299C31A5A1E814200D81A009B4BEF
:1029C0001A608C4B19681E235343994A9B18CB619C
:1029D0008BE701F0E9FA8023E26BDB0213430390FB
:1029E000E363E26D8F4B03201A4028231343E36512
:1029F00001F02AFB0320A56E01F026FBA36E032045
:102A0000DB03DB0B019301F01FFBA76EED03FF035C
:102A1000ED0BFF0B874AAB18C22B2ED8019B9B18DE
:102A2000C22B2AD8BB18C22B27D8019B2A009D4253
:102A300000D21A00019B9D4200D91D003B00974225
:102A400000D21300BD4200D93D005B1B122B14D8ED
:102A50000C2233681420934333603368764A134062
:102A6000336001F0F1FA0821A36EE26DDB038A43C3
:102A7000E265724ADB0B136085E7032001F0E4FA9C
:102A8000A36EDB03DB0B059301F08EFA039B039926
:102A9000C21A531E814200D81300694A93421BD9BF
:102AA000FF23356864492D0A1D4032686B1C1B06E4
:102AB0000A401B0C134333600C23326800209A43F6
:102AC000083B1343336001F097FA5E485E4BA84021
:102AD000984205DCFEF736FF019D0197059F99E7B7
:102AE0005A48F7E700235A4E33608023226CDB02FA
:102AF00013432364636C03202B43636401F0A4FA43
:102B00003368013333608023626C5B021343636478
:102B100005230193E26D434B03201A404D4B1343B1
:102B2000E36501F091FA0821A26EE36D434F8B43F8
:102B3000E3653B6802394B43D203D20B9A420CD86F
:102B40009B1A3B2B0BD8E36D43490B40E365636C49
:102B50000B406364414B1A6028E7D31AF1E7019BED
:102B6000013BDBB20193002BD4D1E36D3A4A134011
:102B7000E365636C134063643368042B07D9BFF3C8
:102B80004F8F374B374ADA60BFF34F8FFEE7636CE6
:102B90000320AB43636401F057FAE26D214B03203D
:102BA0001A4028231343E36501F04EFA0822A36E6E
:102BB000DB03DB0B3B60E36D9343E3659AE707229E
:102BC000E36B1340012B02D1002001F085F9264D63
:102BD000264AAB6802201340AB6001F035FA80232F
:102BE000AA685B001343AB60E0E6C0464A0AFF1FD9
:102BF00000F000405C66FF1F000003400180063DBE
:102C0000BC00034034080000A4000340710200002F
:102C100014100040FFFF3F002810004000E100E0DA
:102C20003075000000FEFEFFC4F000404466FF1F48
:102C30007206000091FCFFFFFF00FFFF4C66FF1FC4
:102C4000E30C0000E88000005F361E0060361E00C6
:102C5000B044FF1F28000100FFFFFEFF4866FF1F72
:102C600000ED00E00400FA053CF00040FFFEFFFF2D
:102C7000694E336888331B6883F3088801F0E4F8F1
:102C800000F018FC654B664A1B68934207D0002091
:102C900001F0B2F90221634A13688B431360FFF716
:102CA00013FE614B614C1878C0B201F08DFA00231D
:102CB000A3600233A3605E4B0120236001F0C4F9DE
:102CC0000323A36001F070F9040001F03DFA050050
:102CD00001F06AF9574B186001F06EF9564B19680C
:102CE000621A531EA14200D213008022D2039342E3
:102CF00001D39B029B0A3268D16AC90700D478E0ED
:102D00004E491C0C09689BB24C4359432402090AE2
:102D1000641803274A49FC3293680A6849489B1A99
:102D2000494A4A4E12684A499B18414A34609A18E7
:102D30003B400193036892089C46019B0A606344F0
:102D40000360042B03D901323B400A6003600B6827
:102D50004049E418200001F0CFF83F4F3D493B685F
:102D6000C3183B602000019301F016F93B4C20682A
:102D7000081838492060884205D9019B01333B601F
:102D800001F00AF9216001F0FFF9354B1B78002BA7
:102D90000ED001F0D9F93168324B4A1B1B6812186A
:102DA0009A4233D2591A4919091A2F4801F094F955
:102DB0002E4C237A002B0FD001F0C6F93168E3685E
:102DC0004A1B1218934224D9591A4919091A28483A
:102DD00001F082F900232372264B83F3088800F068
:102DE000CBFF022001F0A8F8002001F005F900F067
:102DF000EBFFDC0199000234641A5900641A0921BE
:102E00004B438033CB40A408E41882E7FA218900C1
:102E1000CBE71949DBE7C0465C66FF1F0C0AFF1FC2
:102E2000B641210310000040490AFF1F1410004062
:102E3000C4090000100AFF1F340AFF1F380AFF1FD1
:102E4000200AFF1F280AFF1F1C0AFF1F4066FF1FE2
:102E5000240AFF1F710200006008FF1F2C0AFF1FD9
:102E60001C09FF1FE408FF1F00100040740BFF1F28
:102E70003C10004000000020DC050000A022054BB3
:102E800092009B5810B5002B01D0984710BD01F05F
:102E900093F9FBE70000FF1FA122054B92009B580E
:102EA00010B5002B01D0984710BD01F085F9FBE764
:102EB0000000FF1FA222054B92009B5810B5002B6B
:102EC00001D0984710BD01F077F9FBE70000FF1F24
:102ED000A322054B92009B5810B5002B01D09847B8
:102EE00010BD01F069F9FBE70000FF1FA422054BAC
:102EF00092009B5810B5002B01D0984710BD01F0EF
:102F00005BF9FBE70000FF1F70B501F01DF9514BA5
:102F10001860042001F010F800F046FF0400C30719
:102F200002D401F081F970BD00224B4B1A604B4B6B
:102F30001878013804282CD800F0CAFE03231B1F80
:102F40002700200001F018F80128ECD0444C237829
:102F5000042B71D100F0D0FE002806D001F09CF8BF
:102F6000582000F069FF02232370032000F0E4FFE3
:102F7000D9E7200000F078FFE6E7200000F0CCFF62
:102F8000E2E7200000F098FFDEE7200001F00CF9F6
:102F9000DAE700F0D9FF0500012808D1314B1B7892
:102FA000053B012B03D82000FFF768FFCEE72C4B31
:102FB0001B78022B01D0052B20D1022D28D12A4BC2
:102FC0009B7BAB431CD12000FFF766FF254B187895
:102FD0000128BBD16405B9D4234925224B7B034288
:102FE00005D1233A13405A42534126331A000B7D30
:102FF0009342ABD9322000F0CFFEA7E7022D07D1D4
:10300000184B1B78052B11D12000FFF753FFDDE78C
:10301000012D0BD1012B03D12000FFF759FF95E7BC
:10302000062B03D12000FFF761FF8FE7200001F09E
:10303000C3F8022D8AD1C9E7032B04D10B4B987C2E
:1030400000F092FE91E7072B8FD1094B987B00F09F
:1030500063FE8AE79C09FF1F9809FF1F9009FF1F65
:103060002309FF1F1C09FF1FA60BFF1FBC0BFF1F1F
:10307000D40BFF1FFA210A4B0A4A49001A640A4A74
:103080005A500A4A04395A50094A08319A64094A7E
:103090005A50094A5C315A50084ADA667047C046AD
:1030A0000000FF1F7927FF1F7528FF1F2928FF1F1A
:1030B0008123FF1FE926FF1F011EFF1FD51DFF1FD4
:1030C00010B500F0EDFD10BD8023F7B59C46264BF2
:1030D000264F01932649274A274D284C284B022882
:1030E0001AD1604638600868264E30408026360384
:1030F0003043086001990978002909D11660224AF5
:103100002A60224A2260E02219689143A03A1BE01B
:103110008021C9021160F2E766463E600F68194ED1
:103120003E408027FF023E430E6001990978002946
:103130000DD1176001280ED1154A2A60154A226068
:10314000E02219689143C03A0A431A60F7BD802112
:1031500089021160EEE7E0210F4A02432A600F4A1C
:1031600022601A688A43F0E74B0AFF1FE000034021
:10317000D80003409000034000000340500003408B
:1031800040000340FFFFE3FF0280063D8045082228
:103190000180063D8066082200800698805508223E
:1031A000F8B51E4B80261A680020140034403242C5
:1031B00032D11A681A4F32431A6001223B68063036
:1031C00093433B6000F040FF0122164D2B681E43E5
:1031D0002E603B680A2613433B608027BF00124BDA
:1031E0001B683B4211D1013EF6B2FF2E09D17E226F
:1031F0000E4B1C682B68E40B1440934323432B6055
:1032000005E0082000F020FFE9E7002EEFD1802242
:103210002B68600893432B60F8BDC046C4F00040A3
:103220005CF0004018F0004068F0004060F00040A2
:1032300010B500F0E9FD01215820034A00F064FEBA
:10324000FFF7AEFF10BDC046600AFF1F10B5782221
:103250000021034800F0E8FD00F066FE002010BDEC
:103260006469FF1F70B5040000F0F6FE00230C2017
:103270000B4A010059438D18515C00290DD0A14221
:1032800008D1012300246B7000F0FEFE00F0D4FF93
:10329000200070BD01330A2BEBD11224F6E7C046A3
:1032A0006469FF1F70B5040000F0D6FE002319000A
:1032B0001D000D4A1078002806D0A0420CD1557090
:1032C00001310C320A29F5D1002B0AD100F02CFE75
:1032D00000F0B2FF002070BD5078461EB0411B18B0
:1032E000EEE700F0D1FEF3E76469FF1FF7B50400D5
:1032F0000C20002384460E4D019267465F43E85D33
:103300007E19A04212D000280BD10A4B9C4662467F
:103310001B7808331370019B70707C557160B3602B
:10332000FEBD01330A2BE8D10320F9E70720F7E7B8
:103330006469FF1F6069FF1F8020F8B5484BC00516
:103340001B68C1248360474BFF251A680123134380
:103350004361454BA4001A68444B40211A60444B1A
:103360001A68444B1A60444B1A59AA431A51C52291
:1033700092009E58AE433143802699509F583F4952
:10338000F6010F403E439E509E5880273602360A73
:103390003043985080201A5900020A4002431A51C3
:1033A00004341A59364E3F04324080263A431A51AB
:1033B0001A5936061202120A32431A5108341A599F
:1033C00080260A4002431A51C32292009F58B446F5
:1033D000AF4337439F509F58294E0F4007439F509C
:1033E0009F58374080263604374380269F509F5889
:1033F00036063F023F0A37439F50C0221F59AF4352
:103400003A431A511A591202120A1643C6221E5181
:1034100092009C58AC4365462C439C509C58002518
:103420000C4020439850C72080001A58154C11407A
:10343000C02212020A431A50134B1B78DB08AB421E
:1034400001DC0020F8BD2378002B06D0A368002BF8
:1034500000D0984701350C34EEE71220F2E7C04661
:103460004845FF1F4445FF1FB0F000405C69FF1F47
:10347000B4F000405869FF1F00E100E0FF00FFFFCB
:10348000FFFF00FF6469FF1F6069FF1F030010B5A5
:103490001F2809D8072200201340072404490A786E
:1034A000A24313430B7010BD00230620F5E7C0466E
:1034B0006069FF1F034A0449136800200B40136032
:1034C0007047C0461CF00040FFFFC1FF054B064996
:1034D0001B780A6805485B0702401B0B134300205A
:1034E0000B6070476069FF1F1CF00040FFFFC1FFC9
:1034F00070B50C25FFF7EAFF0A4B1C780A4BE4086D
:103500006543ED18002C01D1200070BD2B78002BF5
:1035100006D06B68002B00D09847013C0C3DF1E7CA
:103520001220F2E76069FF1F5869FF1F07B50422E8
:10353000074801A900F034F9019B013305D180232C
:10354000044ADB0411680B43136000200EBDC04623
:103550001C18001114F00040F0B505002026184B8F
:1035600087B00493049B002B03D11124200007B0E3
:10357000F0BD002102220B0001910091052000F016
:10358000B3FD02230F490A681A42FCD10596059C37
:10359000631E0593002CFAD10B4A1368002BFCDA4A
:1035A0000F276F440121380000F026FC3B782B42A6
:1035B000DCD0052000F048FD049B013B0493D1E7DB
:1035C000FFFFFF0790C8004000C8004007B500F0AB
:1035D00043FD80220821D205936A0191002B01D17D
:1035E0000739916202210C4A11600199481E01902D
:1035F0000029FAD103311160053101910199481E6A
:1036000001900029FAD11160002B02D18022D2054D
:10361000936200F011FE07BD00C00040F0B52D4CD4
:1036200089B02378002B4FD1FEF76CF902232A4F83
:1036300003903A681A42FCD120230693069B5A1E37
:103640000692002BFAD1254E3368002BFCDA0120BC
:10365000FFF782FF011E02D0112009B0F0BD030068
:1036600003220190009005AD9F2000F03DFD032155
:10367000280000F0C1FB02233A681A42FCD1202343
:103680000793079B5A1E0792002BFAD13368002B31
:10369000FCDA0120FFF760FF0028DDD10398FEF778
:1036A00045F9AA786B7811041B020B4329780B4368
:1036B00063601300113B0A49052B07D8012393408F
:1036C000A3600B60012323700020C6E780231B0347
:1036D000F6E7C0463045FF1F90C8004000C80040D4
:1036E0009808FF1F1E4B30B55A6818781D4B85B0DF
:1036F000D31859424B4101210093002300F074FB81
:10370000194B1A4A02259A6300221A6510325A652B
:103710008022C4219D65164B1648D202DA678900C3
:103720004258154B80241A4080231B0413434350F6
:10373000642341200393E40500F078F9402000F071
:1037400075F96562039D6B1E0393002DFAD1032367
:103750006362FFF73BFFA562FFF760FF05B030BD76
:103760003C45FF1F95FFFEF700C80040050001FF24
:1037700004E100E000E100E0FFFF00FF10B5064BB0
:1037800018705960FFF7AEFF00211320034AFFF7BE
:10379000ADFD002010BDC0463C45FF1FE536FF1FB4
:1037A000F0B5040085B003920291FEF7ABF88822D1
:1037B00063035B0B52051A438023DB059D6A80235C
:1037C000274F0092BA68002601901B039A420CD939
:1037D000F82326001B041E401C4206D08022214BE9
:1037E00052025E6219680A431A60002D0BD100F084
:1037F00033FC02221C4B1A608023DB055A62013A1B
:103800009A6200F019FD0023039A934220D1002D03
:103810000AD100F021FC144B03221D608023DB053C
:103820005A629D6200F008FD8023BA681B039A4229
:1038300008D9002E06D000220A4B0C495A621A6899
:103840000A401A600198FEF771F8002005B0F0BD3B
:10385000009A0299D2181278CA540133D4E7C046AC
:103860003045FF1F00C8004000C00040FFFFFEFFC2
:10387000F0B587B0029103920400FEF743F801907F
:1038800000F0EAFB802302250122234EDB05356090
:103890005D629A6200F0D0FC204F3B682B42FCD165
:1038A00020230493049B5A1E0492002BFAD11C4D32
:1038B0002B68002BFCDA0120FFF74EFE002802D017
:1038C000112007B0F0BD2000039A029900F05CFBC4
:1038D000022304003A681A42FCD120230593059B79
:1038E0005A1E0592002BFAD12B68002BFCDA01201E
:1038F000FFF732FE051EE3D100F0AEFB802303226A
:10390000DB0535605A629D6200F096FC0198FEF777
:103910000DF8E0B2D5E7C04600C0004090C80040B6
:1039200000C80040F0B5802687B00400FDF7EAFF2C
:10393000F605B36A02250393029000F08DFB012384
:10394000244F3D607562B36200F076FC224E33680E
:103950002B42FCD120230493049B5A1E0492002B7B
:10396000FAD11E4D2B68002BFCDA0120FFF7F4FD85
:10397000002802D0112007B0F0BD200000F0A4FA0A
:103980000223019032681A42FCD120230593059B43
:103990005A1E0592002BFAD12B68002BFCDA03206B
:1039A000FFF7DAFD041EE5D100F056FB8023032269
:1039B000DB053C605A629C6200F03EFC039B002BDE
:1039C00001D1FFF703FE0298FDF7B0FF6B461879AF
:1039D000D1E7C04600C0004090C8004000C8004089
:1039E00007B5000201910422000A01A9FFF740FF78
:1039F0000EBD000073B5050005240B4AA3005B4211
:103A00009B1819686B46DE1D300000F0DDFA0228B5
:103A100004D133782B55013CEFD276BD052CFCD078
:103A20000128FAD10230F8E7140900111F2807D83D
:103A3000012380228340D20591680B439360704735
:103A40003F2808D80123802220388340D2055169BD
:103A50000B435361F3E75F28F1D8012380224038FC
:103A60008340D205116A0B431362E8E71F2807D889
:103A7000012280218240C9058B6893438B60704787
:103A80003F2808D80122802120388240C9054B698F
:103A900093434B61F3E75F28F1D80122802140383E
:103AA0008240C9050B6A93430B62E8E71F2810D8D0
:103AB00080230200DB05153A1968012A06D8202266
:103AC0009143196019680A431A60704701228240C5
:103AD000F6E73F2811D880230200DB05353AD96884
:103AE000032A06D810229143D960D9680A43DA60C4
:103AF000EBE7012220388240F5E75F28E5D8422332
:103B00008022181A413B8340D205516A9943516281
:103B1000516A0B435362D8E710B50400012813D152
:103B2000A022184992050B685B015B0913430B60E7
:103B3000154B164A19681140154A0A431A6040226B
:103B400019680A431A6010BD0028FCD101000A2040
:103B500000F00AFB21000B2000F006FBC0220A4BFC
:103B6000920019680A4340211A601A688A431A6051
:103B7000B022044912060B685B015B0913430B601A
:103B8000E1E7C04614F000401CF000407F00FEFF5B
:103B900080FD010072B6074A1368013313600422E6
:103BA000054B1A600023054A13608022D20553603A
:103BB000FEE7C0467808FF1FC0F00040C4F0004098
:103BC000044B054A1A60054B1A600022044B1A6028
:103BD0007047C046140AFF1F841E0000380AFF1FEA
:103BE000C4F000400023034A1360034A1360034AF1
:103BF0001360704754F0004040F1004044F1004031
:103C0000002310B5184C8AB0009301932378012B40
:103C100027D06946012000F08FFA002817D1009BB9
:103C200012490293019B06AA0393114B02A81B6839
:103C30000493104B1B68059300F0CEF810220E4938
:103C400006A800F061F8002804D1FF2323700020AB
:103C50000AB010BD0123094A074902A8237000F0E9
:103C6000BBF80120F4E7C0466066FF1F1029001171
:103C7000082900110C290011202900116466FF1F7A
:103C800013B501246946012000F056FA034B009455
:103C90000193FFF7B5FF200016BDC046BB0B000027
:103CA00010B5FFF79FFFFFF7EBFF002802D0024B94
:103CB000984710BDFEE7C046E1A2000002B471467D
:103CC00049084900095649008E4402BC7047C04665
:103CD00002B4714649084900095C49008E4402BC9F
:103CE0007047C04603B47146490840004900095A6C
:103CF00049008E4403BC704701B40248844601BCAD
:103D0000604700BF01D7000001B40248844601BCEF
:103D1000604700BFCD4C010001B40248844601BC9D
:103D2000604700BFC1F7000001B40248844601BCEF
:103D3000604700BF53B9000001B40248844601BC8B
:103D4000604700BF8B52010001B40248844601BCA9
:103D5000604700BF6911010001B40248844601BCFC
:103D6000604700BFE927000001B40248844601BC57
:103D7000604700BF4DF9000001B40248844601BC11
:103D8000604700BF7997000001B40248844601BC37
:103D9000604700BF8D11010001B40248844601BC98
:103DA000604700BF6137010001B40248844601BC8E
:103DB000604700BFBD0B010001B40248844601BC4E
:103DC000604700BFB352010001B40248844601BC01
:103DD000604700BF8552010001B40248844601BC1F
:103DE000604700BFDD3F000001B40248844601BCCB
:103DF000604700BFC56D010001B40248844601BCA4
:103E0000604700BF3D71010001B40248844601BC17
:103E1000604700BFED68010001B40248844601BC60
:103E2000604700BFD9B0000001B40248844601BC1D
:103E3000604700BFB70E000001B40248844601BCD1
:103E4000604700BF7912010001B40248844601BCFA
:103E5000604700BFC9A9000001B40248844601BC04
:103E6000604700BFE512010001B40248844601BC6E
:103E7000604700BF0934010001B40248844601BC18
:103E8000604700BF116E000001B40248844601BCC7
:103E9000604700BF9D6A000001B40248844601BC2F
:103EA000604700BFA9D8000001B40248844601BCA5
:103EB000604700BF51B8000001B40248844601BC0D
:103EC000604700BFF535010001B40248844601BCDB
:103ED000604700BFA96F010001B40248844601BCDD
:103EE000604700BFEDA5000001B40248844601BC54
:103EF000604700BF19FA000001B40248844601BCC3
:103F0000604700BF090E000001B40248844601BCAE
:103F1000604700BF0167010001B40248844601BC4C
:103F2000604700BF0534010001B40248844601BC6B
:103F3000604700BFADAE000001B40248844601BC3A
:103F4000604700BF1907010001B40248844601BC64
:103F5000604700BFDD0C010001B40248844601BC8B
:103F6000604700BFC1A5000001B40248844601BCFF
:103F7000604700BFE94C010001B40248844601BC1F
:103F8000604700BF0134010001B40248844601BC0F
:103F9000604700BF9573010001B40248844601BC2C
:103FA000604700BF090E000001B40248844601BC0E
:103FB000604700BF156B010001B40248844601BC94
:103FC000604700BFC166010001B40248844601BCDD
:103FD000604700BF9938001101B40248844601BC13
:103FE000604700BF8512010001B40248844601BC4D
:103FF000604700BFF9ED000001B40248844601BCEF
:10400000604700BF016C010001B40248844601BC56
:10401000604700BF8944000001B40248844601BCE7
:10402000604700BFC115010001B40248844601BCCD
:10403000604700BF75F8000001B40248844601BC27
:10404000604700BFE9D4000001B40248844601BCC7
:10405000604700BF0189000001B40248844601BCEA
:10406000604700BF75A9000001B40248844601BC46
:10407000604700BF5976010001B40248844601BC84
:10408000604700BFE9F6000001B40248844601BC65
:10409000604700BF21A9000001B40248844601BC6A
:1040A000604700BF6DF6000001B40248844601BCC1
:1040B000604700BF79B6001101B40248844601BCD4
:1040C000604700BFED6B010001B40248844601BCAB
:1040D000604700BF6D0B010001B40248844601BC7B
:1040E000604700BF2D6C010001B40248844601BC4A
:1040F000604700BF496D010001B40248844601BC1D
:10410000604700BFF90D010001B40248844601BCBC
:10411000604700BF2144000001B40248844601BC4E
:10412000604700BFA1AF000001B40248844601BC53
:10413000604700BFBD5C010001B40248844601BC79
:10414000604700BFE1AC000001B40248844601BCF6
:10415000604700BFC95C010001B40248844601BC4D
:10416000604700BFF9A6000001B40248844601BCC4
:10417000604700BF8DA2001101B40248844601BC13
:10418000604700BF71B0000001B40248844601BC22
:10419000604700BFD544010001B40248844601BC19
:1041A000604700BF8D82000001B40248844601BC14
:1041B000604700BFF935010001B40248844601BCE4
:1041C000604700BFE917010001B40248844601BC02
:1041D000604700BF8914010001B40248844601BC55
:1041E000604700BF85C1000001B40248844601BC9D
:1041F000604700BFE90B010001B40248844601BCDE
:10420000604700BF0D52010001B40248844601BC62
:10421000604700BF8937010001B40248844601BCF1
:10422000604700BFCD0C010001B40248844601BCC8
:10423000604700BFDD0A010001B40248844601BCAA
:08424000604700BF9DA90000CA
:1042480002000000CEBF00110100000080BD001177
:1042580002000000CABF0011010000008842FF1FD1
:104268000200000088BD001101000000A063FF1FCC
:1042780002000000C8BF0011030000001463FF1F04
:104288001200000002000000CEBF00110100000073
:10429800C8BD001102000000CABF001101000000E3
:1042A800C5BD001102000000D2BD001103000000CE
:1042B8004F63FF1F02000000C8BF00110300000089
:1042C8006463FF1F02000000CABF00110100000064
:1042D800C4BD001102000000D0BD001103000000A1
:1042E8002563FF1F02000000C8BF00110300000083
:1042F8004663FF1F02000000CEBF0011010000004E
:1043080008BE001102000000CABF00110100000031
:10431800D143FF1F020000001ABE00110100000077
:1043280003BE001102000000CABF00110100000016
:10433800D043FF1F0200000018BE0011010000005A
:104348006C63FF1F02000000CABF001101000000DB
:10435800CF43FF1F0200000016BE0011010000003D
:10436800F3BD001102000000CABF001101000000E7
:10437800CE43FF1F0200000014BE00110100000020
:10438800EEBD001102000000CABF001101000000CC
:10439800CD43FF1F0200000012BE00110100000003
:1043A800E9BD001102000000CABF001101000000B1
:1043B800CC43FF1F0200000010BE001101000000E6
:1043C800E4BD001102020202020200000000000027
:1043D80016150000214C0011E74B00115CBE0011BE
:1043E800900118001800FFFF0701020304050602E8
:1043F80001060000000000000000000000000000AE
:1044080000000000000000000000000000000300A1
:1044180002000000CEBF001101000000DCBE001148
:1044280002000000CABF0011010000008844FF1FFD
:1044380002000000E6BE0011010000009A63FF1FA1
:1044480002000000C8BF0011030000000866FF1F3B
:1044580002000000CABF0011010000008844FF1FCD
:1044680002000000E4BE0011010000009C63FF1F71
:1044780002000000C8BF0011030000000066FF1F13
:1044880012A6A6A6000000000000000016150000F5
:104498000001000000000111FFFF000050485936DC
:1044A8000000000000000000010000006DBE0011C7
:1044B8000B000500F7000000B400002800280028C1
:1044C8003075A000A000A000A00000080008E001CE
:1044D800F000100010001000100010001000500034
:1044E8005000500010001000D0070000000000002D
:1044F8000F0001000500307507001000010081FF62
:1045080000000000FF000000757400117D720011AA
:104518000D700011FFFF0100FF000000919E0011C7
:104528000D9C0011259B00110000000000000000F8
:1045380000000800040000003B0001085902E001E7
:1045480088212800FF00000002000000CEBF0011F3
:104558000100000094C0001102000000CABF001151
:1045680001000000CD45FF1F02000000C6BF00117A
:10457800010000001C6AFF1F02000000CABF0011F2
:1045880001000000CC45FF1F02000000C4BF00115D
:1045980001000000CA45FF1F02000000CABF001149
:1045A80001000000C845FF1F02000000C2BF001143
:1045B80001000000C045FF1F18001800000090010E
:1045C800020000030202000002000000CEBF00113A
:1045D80001000000A8C0001102000000CABF0011BD
:1045E800010000001046FF1F02000000C0BF0011BC
:1045F800000000000000000002000000C8BF001119
:0A460800030000003C6AFF1F20FFC2
:040000051FFF184180
:00000001FF
